:020000040800F2
:104000000050002039DA0008D5B10008D9B1000805
:10401000DDB10008E1B10008E5B1000800000000D2
:10402000000000000000000000000000EDB10008EA
:10403000E9B1000800000000F1B10008D1830008D8
:10404000F5B10008F9B10008FDB1000801B200089F
:1040500005B2000809B200080DB2000811B200084C
:1040600015B2000819B200081DB2000800000000D7
:104070000000000000000000000000000000000040
:1040800000000000000000003DB2000841B200083E
:1040900051B2000861B2000871B2000881B2000894
:1040A00085B2000889B200088DB2000891B20008FC
:1040B00095B2000899B200089DB20008A1B20008AC
:1040C000A5B20008A9B20008ADB20008B1B200085C
:1040D000B5B20008B9B2000899810008C1B2000861
:1040E000C5B20008C9B20008CDB200080000000047
:1040F00000000000000000000000000000000000C0
:0C41000000000000000000005FF800005C
:1041100030BF704720BF704740BF7047BFF36F8FFD
:104120007047BFF34F8F7047BFF35F8F704701DF5A
:104130007047EFF31480704780F31488BFF36F8FDC
:104140007047EFF30980704780F309887047EFF3F9
:104150000880704780F30888704772B6704762B66F
:10416000704771B6704761B6704780F31188704729
:10417000EFF31280704740BA704700BA70470000F2
:1041800037B508F02BF94E4B00254FF480301D70E9
:1041900008F044F908F0A8FA0128044626D11020B6
:1041A00007F006FC284608F089F9284608F09AF935
:1041B000284608F08DF94FF480304FF4802108F044
:1041C00059F9204608F062F9392008F077FA0028FA
:1041D000FAD0012007F0D4FB012008F05DF908F0C7
:1041E00065F90428FBD1364B01221A700420012105
:1041F00008F01AFA03238DF80630153301A9314867
:104200008DF807304FF48073ADF8043007F004FEEA
:10421000062008F04DFA0120014608F005FA4FF497
:1042200080414FF0006007F0FBFF4FF4407007F053
:1042300059FF00F085F900F089FA2349234A244BFD
:104240001160244A244C136001222270234A244D19
:10425000136000F0B9F804F017F904F0EBF803F07C
:10426000C9FE00F041F8287803F0F6FFE87803F083
:104270004FFF23780BB104F037FC05F097F906F0F7
:104280007BFD01F009FB04F04BFC05F0D5F9154B63
:104290004FF480625A6104F0C7F803F0FDF805F0AE
:1042A000D9F904F04FFC00F0CBF800F0BBF800287F
:1042B000F3D005F07BF901F0EFFA05F0BDF9ECE77A
:1042C000B00B00200008014089890008C00B0020C5
:1042D000CD830008500B0020D00A0020F00A0020F7
:1042E00004000020000C0140114B82B01B78E3B1A8
:1042F000104B4FF400725A61002301E0019B01331F
:104300000193019A4AF69B539A42F7D9094B4FF40D
:1043100000721A61002301E0019B01330193019AAD
:104320004AF69B539A42E3D8F6E702B0704700BFC3
:10433000FC0A0020000C014010B1012805D101E069
:10434000042200E01022014B5A617047000C01402A
:1043500010B1012805D101E0042200E01022014B38
:104360001A617047000C014038B50546002455FA23
:1043700004F2E3B212F0010F184602D0FFF7E8FF93
:1043800001E0FFF7D9FF0134082CF0D138BD00BFA0
:1043900018B1012806D0002008E0054BD868C0F30A
:1043A000800003E0024BD868C0F30010704700BFE4
:1043B000000C014008B1002003E0024B9868C0F3F4
:1043C000402070470008014062B6704772B67047DF
:1043D00018B9024B4FF480625A617047000C0140DB
:1043E00018B9024B4FF480621A617047000C01400B
:1043F00020B1054B4FF400521A6103E0024B4FF419
:1044000000525A61704700BF00100140044B1878F9
:104410000138C0B201288CBF00200120704700BFC6
:1044200028020020044B1878012801D0002001E068
:1044300002221A70704700BF280200200020704737
:10444000082008B504F00CF8592804D9064B1A784E
:104450004AB9013206E0082004F002F8542802D8D4
:10446000014B00221A7008BD2802002008B503285D
:1044700003D8DFE800F0040D1217002016E000203A
:1044800003F0EEFFB0F5006F94BF002001200DE0B7
:10449000074B9868C0F3801008E0054B9868C0F39C
:1044A000C01003E0024B9868C0F3401008BD00BF85
:1044B000000C014038B500242546E0B2FFF7D6FFD6
:1044C00020B10123A34043EA0505EDB20134082CD5
:1044D000F3D1284638BD00BF10B50446C0B1002056
:1044E00006F0BEFA0221002006F042F9421E00202A
:1044F000014606F0EFF900200246014606F012F9E7
:104500006821002006F034F940F00802002005E0A0
:10451000682106F02DF920F008022046682106F0F7
:10452000D9F910BD08B510B107F084FE01E007F01D
:1045300089FE08BD08B5C90804F0A2FC08BD00BF8B
:104540002DE9F745DFF8308101AD0420012108F0A5
:104550006BF803241026404642F213032946ADF8B7
:1045600004308DF806408DF8076007F055FC1123E4
:10457000C8F8103002233E4F40464FF0040AC8F8F6
:10458000143029464CF20063ADF804308DF8064033
:104590008DF807A007F040FC0820012108F044F83E
:1045A000384641F614632946ADF804308DF80640CC
:1045B0008DF8076007F030FC4FF4F0533B61142393
:1045C00038467B6129464FF4F473ADF8043008F5A2
:1045D00000688DF806408DF807A007F01DFC3046F6
:1045E000012108F021F84FF40057404629468DF884
:1045F0000760ADF804708DF8064007F00DFC4CF232
:10460000000340462946C8F81070ADF804308DF814
:1046100006408DF807A007F0FFFB0121154807F0C1
:104620008BFC00231A461946134C4FF40055656164
:104630002046A468013314F4804F4FF40054046101
:10464000806808BF013110F4804F18BF01320A2B77
:10465000EAD10A2903D10A2A01D1012200E000226D
:10466000064B07481A70012107F066FCBDE8FE857D
:10467000000C01400004300000080140FC0A00204A
:1046800000023000012870B504460D46164608D0D9
:1046900002D302284FD107E0284B4FF480525A61D1
:1046A00007E01022264B02E0244B4FF400625A61CF
:1046B00010E02448022108F019F90028F9D0294611
:1046C000204808F0B7F81F48012108F00FF900282A
:1046D000F9D00FE01C48022108F008F90028F9D0B1
:1046E0002946194808F0A6F81748012108F0FEF8F5
:1046F0000028F9D096B1012C08D002D3022C1AD18F
:1047000007E00E4B4FF480521A610DE010220C4B63
:1047100002E00A4B4FF400621A6107E0012C05D059
:1047200002D3022C07D101E0064800E0064808F059
:1047300083F8C0B200E0002070BD00BF000C014053
:104740000008014000380040003001402DE9F04FE2
:1047500001218BB04FF4804007F074FF494C0120D9
:1047600009AF014607F060FF03264FF0180B204603
:1047700039464AF20003DFF81491ADF824304FF0C7
:10478000040A8DF826608DF827B007F045FB204617
:1047900039464FF480430DF11008ADF824308DF800
:1047A00026608DF827A007F037FB4FF482730024B2
:1047B00002224FF4007C012548464146ADF81230F4
:1047C0004FF00803ADF81620ADF81AC00392CDF8EB
:1047D00008C0ADF81C30ADF81040ADF81440ADF88D
:1047E0001850ADF81E40ADF8204007F0AFFF484626
:1047F000294607F0E7FF29464FF4805007F014FFE1
:1048000009F550492846214607F096FB48463946A7
:104810004FF0A003ADF824308DF827B08DF8266056
:1048200007F0FAFA484639464FF04003ADF8243015
:104830008DF826608DF827A007F0EEFA039ADDF8D0
:1048400008C04FF482734146ADF812300E484FF065
:104850001003ADF81620ADF81AC0ADF82040ADF841
:104860001040ADF81440ADF81850ADF81C30ADF85C
:104870001E4007F06BFF0448294607F0A3FF0BB06A
:10488000BDE8F08F000C01400030014000380040CE
:10489000014B1878704700BF2C0200202DE9F84525
:1048A000054614460E4600294BD0002849D08142C7
:1048B00047D04FEA42185FFA88F848F006073946B1
:1048C000002005F055FF48F00C018246002005F05D
:1048D0004FFF804628460BF055F9054630460BF051
:1048E00051F9014628460BF059FA064650460BF09E
:1048F00049F931460BF052FA0BF062FB054640468F
:104900000BF040F931460BF049FA0BF059FB0E4918
:10491000002814BF80464FF001083046002D08BF24
:1049200001250BF025FB18B14146204606F09AF907
:1049300039462A46002005F0CDFF044BE418012338
:104940002371BDE8F88500BF0000A0412C020020C3
:1049500070B50D4D044645192B799BB1C6B20B4B72
:10496000710141F0060153F8202001F0E60100201A
:1049700006F044F8064B304653F8241006F072F95E
:1049800000232B7170BD00BF2C020020CC0A002038
:10499000C806002073B5A34CA578002D40F0EE8228
:1049A0006378A42B00F041825AD8842B00F0C58094
:1049B00026D8062B00F00C8110D8022B00F0BD8009
:1049C00006D8002B00F0A980012B40F0D582AAE088
:1049D000042B00F0D68000F2E680CCE0802B00F0C3
:1049E0009C8007D80C2B00F00B810D2B00F0288148
:1049F000072B78E0822B00F0358100F2C28092E034
:104A0000942B00F0FD8016D88A2B00F03B8108D84B
:104A1000862B00F0C880C0F0AE80872B40F0AC82BF
:104A20002AE18D2B00F04D81932B00F009818C2B16
:104A300040F0A2823AE1A02B00F0E28109D8992B44
:104A400000F062819A2B00F07481952B40F09482E3
:104A50003DE1A22B00F0DE81724C00F2E181D4E155
:104A6000B32B00F05D8227D8AB2B00F01F8211D84A
:104A7000A72B00F0068206D8A52B00F0E481A62B18
:104A800040F07A82EEE1A92B00F00582654C00F23D
:104A90000882FBE1AF2B00F02E8206D8AD2B00F090
:104AA0001E82604C00F221820EE2B12B00F02D82BA
:104AB0005C4C00F2308223E2C32B00F0608115D8F9
:104AC000B82B00F0548208D8B62B00F0368200F2E2
:104AD0004982B52B40F0508227E2C12B00F0428181
:104AE00000F24581C02B40F047827CE0D42B00F0DF
:104AF000638109D8C82B00F04981CC2B00F0548188
:104B0000C72B40F0398263E0D62B00F06181C0F002
:104B10005A81FE2B40F0308262E1424B00205A68FD
:104B20000146DB7804E03F4B00205A68DB78022125
:104B300043EA022205F0CEFE23E23A4C0020E3785D
:104B40006268082143EA022205F058FFE378A17861
:104B50006268490143EA0222002A41F00601B8BF17
:104B6000524201F0E601002005F048FF2E4AA378EA
:104B7000D3180122F9E12B4B00205A680A21DB7877
:104B800075E0284C0020E3786268062143EA02229F
:104B900005F034FFE2786068A37842EA0020224AF8
:104BA00022499A180FE01F4C0020E378616843EA1D
:104BB000012106F057F8E2786068A37842EA002005
:104BC000194A1B499A1841F8230000231371D8E1B0
:104BD000144B184AD978184B01201B781070174ACB
:104BE000022B5172DCE00F4B0122D978124B18785E
:104BF000104B1A70114B9972002840F0C281AEE13F
:104C00001421002001AA05F005FE064A9DF8053092
:104C10005168D27852EA012114BF43F0020323F015
:104C2000020365E0440600202C020020CC0A00208C
:104C3000C8060020B80B0020BC0B0020540B00203D
:104C40001421002001AA05F0E5FD9B4A9DF80530DE
:104C50005168D27852EA012114BF43F0010323F0D6
:104C6000010345E0944B00205A68DB78042143EAB5
:104C7000022205F0C3FE84E18F4B00205A680E210A
:104C8000DB78F4E701AE32461421284605F0C2FD78
:104C9000A178E378490141F01401284601F0F401BC
:104CA00032468DF8063005F051FF6AE1824B834AA7
:104CB000DB780020C3F10801C9B2D37204F0FAFB1B
:104CC0005FE17D4B00205A681A21DB78CFE7142181
:104CD000002001AA05F09EFD774A9DF80530516835
:104CE000D27852EA012114BF43F0040323F00403F5
:104CF0008DF80530704B0020997801AA490141F0E8
:104D0000140101F0F401CEE701AC22461821002085
:104D100005F080FD684A9DF805309178D278490108
:104D200002F00F0223F00F0341F0180142EA0303DF
:104D300011E001AC22461821002005F06BFD5E4A0F
:104D40009DF805309178D278490103F00F0341F0C6
:104D5000180143EA021301F0F801224600208DF801
:104D60000530A0E7544BDA78544B1A7209E1524BE4
:104D70005A68DB7843EA0222504B1A6001E1E3787B
:104D8000626843EA02224D4B5A60FAE04A4B4C4AB1
:104D9000D9784C4B01201B781070484A032BD177EF
:104DA00040F0EF800138DAE0434B5A68DB7843EAA1
:104DB0000222424BDA81E4E0E378626843EA0222AD
:104DC0003E4B5A61DDE03C4BDA783C4B9A77D8E0B9
:104DD000394B5A68DB7843EA0222384B9A83D0E099
:104DE000354B364A5968DB7843EA0121052904D856
:104DF00018461373FFF770FBC3E000231373C0E082
:104E00002846E17804F048FBBBE0E178002004F09C
:104E100039FBB6E0284B0020D97804F013FAB0E053
:104E2000E178002004F002FAABE0284603F0C0FE6F
:104E3000E178A37818B9184604F0E0F9A1E0184623
:104E400004F0ACF99DE0002003F0B2FE1A4C20B94A
:104E5000E178A07804F0C6F993E0E178A07804F056
:104E600085F98EE0002003F0A3FE134C20B9E17811
:104E7000A07804F0ABF984E0E178A07804F082F93E
:104E80007FE02846E17804F095F97AE0E1780020A7
:104E900004F09AF875E0084B0020D97804F088F8FF
:104EA0006FE0E178002004F077F86AE02846E178C6
:104EB00004F066F865E000BF44060020540B0020B3
:104EC000B80B0020BC0B0020E178002004F04CF867
:104ED000A1782C4BE27803EBC1035A7151E02A4BC5
:104EE0000020D97803F0E4FF4BE094F90310002090
:104EF00003F0D2FF45E02846E17804F067FA40E08D
:104F0000E178002004F056FA3BE01F4B0020D978EE
:104F100004F044FA35E0E178002004F033FA30E0A0
:104F20002846E17804F016FA2BE0174B5A68DB7834
:104F300043EA0222154B9A6123E0134A114B506851
:104F4000D27842EA0020186010B9597904F00CF8C0
:104F50000D4B0F4A9878125C012A12D1D978FFF7CD
:104F6000E9FA0EE0084BDA78064B1A7109E0284698
:104F7000E17804F04FF904E0032200E00422054B3D
:104F80001A707CBDE00A002044060020540B00206B
:104F9000BC0B0020BC06002013B5AB4B9878002852
:104FA00040F04B825B78A32B00F0D081A74C71D8E6
:104FB000832B00F0F8802ED8082B00F0FE8013D849
:104FC000032B00F0EB8005D8012B00F0DE8000F20F
:104FD000E280D7E0052B00F0E880C0F0E480062BEB
:104FE00000F0E580072B9CE00C2B00F0EF8005D84B
:104FF0000A2B00F0168100F20281FBE0802B00F00A
:10500000C18001D80D2B20E0812B00F0BE80822BC7
:1050100040F0108212E1942B00F0D88018D8872B32
:1050200000F00F8105D8852B00F0B88000F2BD801C
:10503000B1E08C2B00F01C8103D88A2B40F0FA8160
:105040000EE18D2B00F01A81932B40F0F381C7E025
:105050009C2B00F0E6800ED8992B00F01E8103D81F
:10506000952B40F0E7810EE19A2B00F020819B2BDD
:1050700040F0E081C3E0A02B00F05C8103D89D2BC1
:1050800040F0D88199E0A12B00F05881A22B40F08C
:10509000D18157E1B62B00F0C08135D8AC2B00F0A0
:1050A000978115D8A72B00F0808105D8A52B00F09B
:1050B000608100F26C814EE1A92B00F07D81C0F08F
:1050C0007781AA2B00F07C81AB2B40F0B3817BE190
:1050D000B12B00F091810BD8AE2B00F08081C0F095
:1050E0007A81AF2B00F08081B02B40F0A3817FE16B
:1050F000B32B00F08881C0F08281B42B00F087814F
:10510000B52B40F0978185E1C72B50D018D8C12B23
:1051100000F0D68008D8B82B00F08881C0F08181DB
:10512000C02B40F0878145E0C32B00F0CF80C0F05A
:10513000CA80C42B00F0CD80C52B40F07B81CAE033
:10514000D02B00F0E8800ED8CC2B00F0C98003D81B
:10515000C82B40F06F81C0E0CE2B00F0C480CF2B75
:1051600040F06881C1E0D52B00F0DB8003D8D42B60
:1051700040F06081D2E0D62B00F0D680FE2B40F0CC
:105180005981D4E00020014601E00020022105F011
:10519000EFFA606054E10020082101E000200A21BC
:1051A00005F020FBF5E72A4B8EE02A4B36E12A4B2F
:1051B0005B7A34E1284B9B7A31E1002005F0EEF96F
:1051C000214B9B785B0050FA03F310E00020142180
:1051D00001AA05F01FFB9DF80530C3F340031EE153
:1051E0000020142101AA05F015FB9DF8053003F0FD
:1051F000010314E1194B9A68C2F3401213E17C21B8
:10520000002001AA05F006FB0F4B02219A789DF8B9
:105210000630520011FA02F21A420CBF0023012399
:10522000FDE001AA00207C2105F0F4FA064B9DF870
:1052300006209B785B0052FA03F3D8E70020042194
:105240001EE00E21ACE700BF44060020BC06002093
:10525000CC0A0020C8060020540B0020000C01409E
:1052600001AA0020142105F0D5FA9DF80620DAE005
:10527000002003F07DFCC0F1080069E000201A2145
:1052800005F0B0FA64E001AA0020142105F0C2FA8A
:105290009DF80520C2F38002C5E001AA0020182174
:1052A00005F0B8FA9DF8052002F00F02BBE001AA54
:1052B0000020182105F0AEFA9DF805201209B2E091
:1052C000684B1B7AABE0674B1A68ACE0654B5A68D9
:1052D000A9E0654BF8E7654BF6E7624BDA7FA2E0A1
:1052E000604BDA899FE0624BEEE7624A624B1278CC
:1052F000002159600AB101225A60604B5D4A1B7857
:105300000021117023B15C4B5A6842F002025A60CE
:1053100000225A4B93E05A4B1B7880E0514B5A695C
:1053200081E0504B9A7F7EE04E4B9A8B7BE04D4B59
:105330001A7B78E0002003F023FC09E0002003F052
:1053400027FC05E0002003F02BFC01E003F030FC1B
:10535000494B586074E0002003F02AFC464C494B4E
:1053600018B9987803F034FC13E7987803F050FCF0
:105370000FE7002003F01CFC3F4C424B18B9987813
:1053800003F02EFC05E7987803F052FC01E70020BB
:1053900003F00EFC384C3B4B18B9987803F028FC0E
:1053A000F7E6987803F03CFCF3E603F029FCF0E61E
:1053B000002003F045FCCBE7002003F049FCC7E7E1
:1053C000002003F04DFCC3E7002003F051FCBFE7D1
:1053D0002D4B5B7923E0002003F05AFCB8E7002056
:1053E00003F05EFC40B2B3E7002003F06BFCAFE7D4
:1053F000002003F06FFCABE703F074FCC9E600206B
:1054000003F078FCA4E7002003F084FCA0E71F4B26
:105410001A7808E0134B9A6905E01B4B1B68636020
:105420000EE0194B1A79144B5A6009E0002003F082
:10543000C7FB8DE70323237002E00F4B04221A7091
:10544000134B1B786BB10C4B12495A68124B0A6014
:105450001AB91A6842F0080202E01A6822F008023B
:105460001A601CBD540B0020D40A0020780B0020C9
:10547000F80A0020480B0020BC060020EC0A00209F
:105480004C0B002044060020E00A0020DC0A00202B
:10549000B6060020A40600204C06002010B51B4ACA
:1054A0005378142B2DD8917871B95468D078184A54
:1054B0001849927E40EA042041F8230022B31BB32E
:1054C00003F5C270013013E0FF2918D163B94FF41E
:1054D000C3641149204609190422043402F0C2FBB6
:1054E000B4F5CD6FF5D10FE003F5C2700949013075
:1054F00001EB83018000042202F0B4FB04E00422EB
:1055000000E00322054B1A7010BD00BF44060020C6
:1055100004000020500600203C000020BC060020B3
:1055200038B51F4C6578142D36D8A07810F0800F50
:1055300018D010F0010F06D00020022105F018F954
:10554000184B43F82500184B9B7E43B3144B5B78F4
:105550002BB303F5C2701349013001EB83018000C6
:10556000042214E0B0B9022105F002F90E4A0D4BF5
:10557000927E43F8250092B1617881B1A07804222F
:10558000091801F5C270013003EB8101800002F0BF
:1055900069FB04E0042200E00322044B1A7038BDCA
:1055A000440600205006002004000020BC06002015
:1055B00038B56E4CA07808B10422D3E063789A2BFA
:1055C00022D8992B80F09B80822B00F081800BD811
:1055D000062B6ED003D8042B38D0052B0AE0072BFE
:1055E0006DD00C3B012B0CE08C2B75D005D8832B98
:1055F0002CD0862B40F0B5803FE08D2B7DD0933BA7
:10560000022B00F2AE8060E0C72B52D00ED8C12B27
:105610007AD005D8B52B74D0C02B40F0A2804EE0D4
:10562000C22B77D0C32B40F09C8076E0D42B7DD06A
:1056300005D8C82B74D0CC2B40F0938073E0D62BC8
:105640007CD077D3FE2B40F08C807DE0474D00204E
:10565000062105F0E5FAAC780020610141F0060171
:1056600001F0E60105F0BEF8414AAB78D318414A93
:1056700042F8240000221A7176E03C4D00200C21F3
:1056800005F0CEFAAC780020610141F00C0101F088
:10569000EC0105F0A7F8AB78374A354942F8240009
:1056A00018465B1852F8201000221A7105F0DAFA39
:1056B0005AE0492002F0BEFA304B587254E04A20BA
:1056C00002F0B8FA2D4B98724EE00020142100E051
:1056D000042105F0A5FA47E04B200122284902F0F9
:1056E00085FAA378254A184602EB4313D97AC1F10B
:1056F0000801C9B203F0DEFE36E01A21E9E71821FD
:10570000E7E758201F4913E0482002F093FA1B4BAB
:10571000187229E0402019490AE044201A4907E09C
:105720005F201A4908E04E20194909E01949542020
:10573000042206E018495E20012202E017495C209D
:10574000022202F053FA0FE04C200122144902F029
:105750004DFAA278094B03EB4213187BFEF7BCFE0F
:1057600002E003220F4B1A7038BD00BF4406002030
:105770002C020020CC0A0020C8060020540B002078
:105780005F0B00206C0B0020580B0020730B0020D7
:10579000620B0020680B0020720B0020700B0020B1
:1057A000600B0020BC06002010B51E4A5378142B55
:1057B00034D89278AAB91C4A1C4952F823201C4BB1
:1057C0004A601B78002B2CD01A491B4B0A601AB96F
:1057D0001A6842F0080202E01A6822F008021A6011
:1057E0001FE0FF2A18D163B94FF4C3641349204660
:1057F00009190422043402F0F9F9B4F5CD6FF5D19A
:105800000FE003F5C2700849013001EB830180000D
:10581000042202F0EBF904E0042200E00322034B2F
:105820001A7010BD4406002050060020BC0600205F
:10583000B6060020A40600204C0600203C000020F4
:1058400037B5134C657815B1012D1DD112E0042236
:1058500040F2FB7001A902F0C9F9E378626843EAFB
:105860000222019B9A420B4B02D101225A600EE0A8
:105870005D600CE0A3782A2B06D1E11C40F2FB709E
:10588000042202F0EFF902E0024B03221A703EBD3F
:1058900044060020BC060020374938B500230B60C1
:1058A0003649374A0B60374993740B609360D36075
:1058B00013745374344A4FF0FF3142F82310334AC3
:1058C0000024D45401332F2BF4D10731204604F0A7
:1058D0004FFF2F4B0C211860204604F049FF2D4D3F
:1058E0002D4BE97A1860C1F108012046C9B203F0D6
:1058F000E1FD287BFEF7F0FD284B0022E250043446
:10590000B4F5806FF8D1264B9B7E5BB104F506742D
:105910002449204609190422043402F067F9B4F539
:10592000CD6FF5D11E4BDB7E5BB94FF4A7641E49EA
:10593000204609190422043402F058F9B4F5C36F63
:10594000F5D1174B1B79012B03D0112B01D0212B43
:1059500001D1012200E00022094B83F8D020104B36
:105960005B7D23B1FEF752FD08B1012200E0002269
:10597000034B83F8D12038BDA4060020C4060020C4
:105980002C0200204C06002040020020CC0B0020FE
:10599000CC0A0020540B0020C8060020CC060020B2
:1059A000040000203C0000209401002008B50B4BAF
:1059B0005A7892B9997881B95A68DB7843EA022219
:1059C00040F2D2439A4208D140F2FF7002F0C8F987
:1059D00002F08AFA0120FEF7A5FD08BD440600206A
:1059E00010B59A4B9A78022A00F04D81032A00F0F4
:1059F0005381002A40F0E3815A784D2A00F0B680A6
:105A000023D8452A70D00ED8422A56D005D8402A2D
:105A100045D0412A40F0D18146E0432A53D0442A60
:105A200040F0CB8156E0482A7BD005D8462A61D089
:105A3000472A40F0C2816AE04B2A00F0848000F2DD
:105A40008E80492A40F0B98171E0542A00F0D48058
:105A500011D8512A00F0AA8006D84F2A00F08C8075
:105A6000502A40F0AA819AE0522A00F0B180532ACD
:105A700040F0A381B6E0832A00F0DF8006D8552AE3
:105A800000F0C780572A40F09881CFE0852A00F0C7
:105A9000ED80C0F0E380FF2A40F08F81EFE06B4B98
:105AA00040F2FF70D97805E0684B694ADB78002046
:105AB0001946137002F054F984E1DB78644A194600
:105AC00001205370F6E7614B614ADB7804201946E8
:105AD0001371EFE75D4B5E495A68DB781C2043EA9F
:105AE000022341F81C3F0EE0DB78594A1946052095
:105AF0005371DFE7554B56495A68DB780C2043EA6F
:105B0000022341F80C3F042202F0ACF85AE14F4B5B
:105B10004F495A68DB78082043EA022341F8083FDE
:105B2000F1E7DB784A49262001F8263F6FE0474A33
:105B3000474BD27812B1474901224A60DA75444B8B
:105B40001720D97DB6E7414B414CDB78032019463D
:105B5000E37002F005F9E07802F0DAFA32E13B4B4B
:105B60003B4ADB78022019469370A3E7DB78384A7A
:105B70001946152053759DE7344B354CDB781920B9
:105B80001946637602F0ECF8607E10F0010002D056
:105B90000020012100E0014604F01EFF12E12B4B22
:105BA0002B4ADB7816201946937583E7284A127D25
:105BB00012F0010F05D0DB7813F0010F01D102F0D4
:105BC00093F9224B224ADB7814201946137571E7AA
:105BD0001E4B1F495A68DB78202043EA022341F814
:105BE000203F90E7194B1A495A68DB78102043EAA6
:105BF000022341F8103F86E75A68DB7843EA022225
:105C0000012A00F2DC8012491A2001F81A3F012211
:105C10007AE70E4B5A68DB7843EA0222012A00F247
:105C2000CE800B491B2001F81B3FF0E7074B0849CA
:105C3000DB78272001F8273FE9E75A68DB7843EA59
:105C40000222054BC3F8D420BCE000BF440600206C
:105C500004000020BC0600202C0200205A4B5A6889
:105C6000DB7843EA0222594B1A60ABE0564B5A6884
:105C7000DB7843EA0222564BC3F8D820A2E0524B0D
:105C8000DA78544B9DE05868D9785A78524B41EAFB
:105C9000002143F8221095E05A78272A59D00ED8CF
:105CA000022A33D004D8CAB1012A40F0868021E00C
:105CB0001B2A3ED01C2A44D0092A7ED132E02B2A4E
:105CC0005FD005D8292A50D0D978444A54D847E023
:105CD0002D2A64D05CD32E2A6FD167E05A68DB7816
:105CE00043EA02223D4B1A6002F09EFB384BC3F898
:105CF000DC0067E05A68DB7843EA0222374B5A60DF
:105D000002F092FB324BC3F8E0005BE05A68DB78AC
:105D100043EA0222314B9A6002F086FB2C4BC3F817
:105D2000E4004FE05A68DB7843EA02222B4BDA604A
:105D300048E05968DB78002043EA012104F046FF7F
:105D400040E05968DB78002043EA012104F012FFAB
:105D500038E05A68DB7843EA0222204B1A6131E0CE
:105D60005B6841EA032151612CE05A68DB7843EA21
:105D700002221A4B9A6125E05B6841EA0321D16156
:105D800020E05A68DB7843EA0222144B1A6219E0D9
:105D90005A68DB7843EA0222104B5A6212E05A68D2
:105DA000DB7843EA02220D4B9A620BE05A68DB78FB
:105DB00043EA0222094BDA6204E0032200E00422F3
:105DC000074B1A7010BD00BF44060020B806002023
:105DD0002C020020B5060020CC0600207C0B002001
:105DE000BC06002008B5824B9A78022A00F0B980E0
:105DF000032A00F0BB80002A40F01E815B78502B04
:105E00006ED022D8462B54D00ED8422B47D005D87E
:105E1000402B3DD0412B40F00D813EE0442B43D040
:105E2000744B754A43D83DE04B2B4DD006D8482BD8
:105E300043D040D3492B40F0FD8042E04D2B49D068
:105E400045D34F2B40F0F68047E0812B5FD010D830
:105E5000542B4ED005D8522B47D0664B664A46D8B5
:105E600041E0572B4BD0802B4DD0552B40F0E2809A
:105E700042E0852B5DD004D8832B53D05D4B55D8A1
:105E80004DE0FE2B64D066D8F02B40F0D3805FE06D
:105E900040F2FF7001F0CEFE9CE0574B59E0564BAC
:105EA0005A78C4E01279C3E0534BDA69BFE0527903
:105EB000BEE0514B85E0504B80E04F4B93F82620DD
:105EC000B5E04D4BDA7D48E04B4BDA78AFE04A4B1A
:105ED0009A78ACE0484B5A7DA9E0474B5A7EA6E041
:105EE000454B9A7DA3E0127DA2E0434B95E01269F9
:105EF0009EE0414B9A7E9AE03F4BDA7E97E03E4B24
:105F000093F8272093E03D4B93F8D1208FE03B4B53
:105F100093F8D120042A14BF0022012287E0374AD7
:105F2000926885E0354BD3F8D42080E0344A12687B
:105F30007EE0324A334BD2F8D8104B4303F540533E
:105F400039332C4923F000404860C2F8D83076E05D
:105F50002D4B1A786BE02D4B1A78003A18BF0122AE
:105F600065E05A782A4B53F8222060E05B78272BB3
:105F700033D00DD8022B20D003D8C3B1012B59D177
:105F800018E01B2B1FD01C2B21D0092B52D117E05E
:105F90002B2B41D005D8292B24D0164B1D4A24D8B1
:105FA0001EE02D2B3ED03AD32E2B43D13DE0194B92
:105FB0001A683CE0174B5A6839E0164B9A6836E08D
:105FC000144BDA6833E0002004F04EFC02E00020BD
:105FD00004F036FC074B586031E00E4B1A6926E09E
:105FE000526925E00B4B9A6921E0D26920E000BF9D
:105FF00044060020BC060020040000202C020020E3
:10600000B80600206D4EC641B00B0020B50600203A
:10601000CC0600207C0B0020124B1A6A07E0114BC3
:106020005A6A04E00F4B9A6A01E00E4BDA6A0E4B93
:106030005A6004E0032200E004220B4B1A700B4B61
:106040001B786BB1084B0A495A680A4B0A601AB9A7
:106050001A6842F0080202E01A6822F008021A6088
:1060600008BD00BF7C0B0020BC060020B606002047
:10607000A40600204C06002010B5154CA07818BBD3
:106080006378012B16D003D3022B124C19D114E0E4
:1060900003F032FFA17839B10F4A937FBBB102EB15
:1060A0004112927F9A4212D10C4B01221A71013A8D
:1060B0000B4B0BE003F028FF09E003F02DFF6060BD
:1060C00005E00323237002E0024B04221A7010BD86
:1060D00044060020BC060020540B00202C020020A7
:1060E000EC0A002037B5504B1A7CA2B94F494868DA
:1060F000CA7842EA0022B2F1FF3F04BF4C4A12685C
:106100000A214A43C3F8E82002F08EF9464B0122E7
:106110001A74C3F8EC00454B5B78042B00F28280C4
:10612000DFE803F003353F4F130002F07DF93E4BEB
:10613000D3F8EC10D3F8E820411A0029B8BF49423F
:1061400091426CD900221A746CE0384B364C987826
:1061500003F0E2FE30B9374A2074136823F01003CD
:1061600013605FE0D4F8E830002B57D002F05CF900
:10617000D4F8EC20D4F8E830821A002AB8BF524292
:106180009A424BD92B4B00211A68217442E000201F
:1061900004F004FA254B244C9D786D0050FA05F567
:1061A0001CE000207C2101AA04F034FB1F4B0222DA
:1061B0009D789DF806306D0012FA05F51A4C1D40C9
:1061C0000EE001AA00207C2104F024FB174A9DF870
:1061D00006309578144C6D0053FA05F515F001055D
:1061E00006D0144B00211A68217422F0100213E02B
:1061F000D4F8E83093B102F017F9D4F8EC20D4F8D1
:10620000E830821A002AB8BF52429A4206D9094B96
:1062100025741A6842F010021A6003E0024B9A6873
:10622000013A9A603EBD00BF2C02002044060020C7
:10623000A40600204C06002008B5184B9A7812B12D
:10624000022A26D106E05868DB7843EA0020FEF7F0
:10625000CFF821E0587807280AD85A68DB7853EA43
:10626000022202D1FEF768F816E0FEF771F813E09B
:10627000FF280CD15868DB7843EA0020B0F1FF3FDB
:106280000ABF074BC0B21878FEF76EF804E003228D
:1062900000E00422034B1A7008BD00BF4406002032
:1062A000A4060020BC06002010B5234B9A78012AD2
:1062B00025D003D3022A214C2AD124E0587808287B
:1062C00002D8FEF7D3F817E00A2801D100220CE02B
:1062D0000B2802D1FEF7B2F80EE00C2808D1184BBB
:1062E0009A6882F40042C2F3C032144B5A6011E043
:1062F000FF280FD1FEF7DEF8104B58600AE05878FF
:1063000002F0AEF8F8E75878FEF742F8606001E076
:10631000042323700B4B1B786BB1084B0A495A6856
:106320000A4B0A601AB91A6842F0080202E01A68B9
:1063300022F008021A6010BD44060020BC060020AE
:1063400000080140B6060020A40600204C060020EC
:1063500010B5204B5A78812A3AD19A78922A37D1AF
:106360009A79A32A34D15A79B42A31D11A79C52A13
:106370002ED1DB78D62B2BD1174B4FF480621A61CC
:1063800002F072FB02F050F8044602F04DF8001BD8
:106390000028B8BF4042B0F57A7FF6DBFEF716F86A
:1063A00005F06EFE002006F09BFB00210B4805F077
:1063B0001DFA0A4805F07AF9094805F04DF905F08B
:1063C00065FA4FF0804007F00FF90020FEF7AAF8B9
:1063D00010BD00BF44060020000C01400800024030
:1063E000002401402DE9F3479D4A9E4DD078516825
:1063F000137840EA01204FF0640C222B85F800C08E
:106400006B70686000F0838554D80F2B00F03E83DA
:1064100024D8072B00F00A8210D8032B00F0F88054
:1064200006D8012B00F0A680022B40F0B187C8E00F
:10643000052B00F0F38100F2F58101E10B2B00F058
:10644000E88205D8092B00F0DC8200F2DE82D4E27B
:106450000D2B00F0138300F21583F3E2192B00F0EB
:10646000BD8412D8152B00F0C98306D8132B00F079
:106470001183142B40F08C8774E3172B00F08E846B
:10648000794B00F29E8400F082BC1E2B00F0D08479
:1064900009D81B2B00F0C484C0F0B0841C2B40F042
:1064A000778700F0C0BC202B00F0C88400F2C984BC
:1064B00000F0C1BC812B00F0D8852ED8412B00F014
:1064C000BA8515D8252B00F0688507D8232B00F056
:1064D0002A85242B40F05C8700F031BD272B00F08B
:1064E0009385C0F06585402B40F0528700F0A0BD39
:1064F000452B00F0AC8506D8432B00F0A28500F2B6
:10650000A38500F09BBD472B00F0A785C0F0A285B6
:10651000802B40F03D8700F0A3BD882B00F047861C
:1065200012D8842B00F0EC8507D8822B00F0B585BB
:10653000832B40F02D8700F0B5BD862B00F0FA8547
:1065400000F2548600F0F1BD8C2B00F0998606D83D
:106550008A2B00F07C8600F28E8600F075BEF22B4E
:1065600000F0E686FF2B00F005878D2B40F01087AA
:1065700000F089BE9378FBB93B4B4FF0010C83F8D8
:1065800004C03A4B00241C70394B21461C70204635
:10659000022204F0C7F82046062140F2FF7204F000
:1065A0002DFA2F4B20465A68DB78082143EA022255
:1065B00004F024FA00F0EFBE2A4B04221A7000F017
:1065C000EABE274DAC78F4B9274B4FF0010C83F8A5
:1065D00004C0264B21461C70254B20461C7002220D
:1065E00004F0A0F82046062140F2FF7204F006FAFB
:1065F0006A68EB78204643EA02225242082104F0FE
:10660000FDF900F0C8BE174B04221A7000F0C3BE9B
:1066100094788CB9154B20461C70154B1C7003F0F8
:1066200073FC20462146022204F07CF82046082113
:1066300004F0F8F900F0AFBE04232B7000F0ABBEFD
:10664000074B9A78002A40F0E4805B78032B00F235
:10665000DB80DFE813F00F0049009400BA0000BFB0
:1066600044060020BC0600202C020020480B00201D
:10667000EC0A0020A64D0020FEF76AF9A54EAB7883
:1066800000246868EA78F454A34E590142EA0022D3
:10669000F45401F0E001204604F01CF9A9782246E8
:1066A000204604F03FF8A9789C4A02EB41139B7FF7
:1066B000002B00F07086002900F06D86927F9A42D0
:1066C00040F069862046FEF743F96A68EB78204679
:1066D00043EA0222214604F0FDF8204621462246E4
:1066E00004F020F800F057BE894D0020FEF730F985
:1066F000AB78884A00245901D454874A41F00201FA
:10670000D45401F0E201204604F032F8EB786E68D0
:10671000A97843EA06268619490101F0E0013246CC
:10672000204604F0D7F82046A978224603F0FAFF65
:10673000A8787A4A7A4902EB40139B7F4E60002B7F
:1067400000F02986002800F02686927F9A4240F0C9
:106750002286FEF7FDF80221204604F009F86A6857
:10676000EB78214643EA02228218204604F0B2F870
:1067700020462146224603F0D5FF00F00CBE644CB3
:10678000E378626843EA0223142B19DC654A00208F
:1067900052F82360FEF7DCF8A37832465D4E002500
:1067A000F5545D4E5901284601F0E001F55404F01E
:1067B00091F82846A1782A4603F0B4FF00F0EBBD1B
:1067C000574B04221A7000F0E6BD514C0020E378CC
:1067D0006268002543EA0222524B53F82260FEF71A
:1067E000B7F8A37832464B4E5901F5544A4E284625
:1067F00001F0E001F55404F06DF82846A1782A462E
:1068000003F090FF00F0C7BD454B03221A7000F063
:10681000C2BD434B04221A7000F0BDBDFEF7BAF8AA
:1068200000F0B9BDFEF7B8FB00F0B5BD907818B127
:1068300004232B7000F0AFBD53789A2B21D8992BED
:1068400080F08480822B6FD00BD8062B4BD003D8DE
:10685000042B3CD0052B0AE0072B4BD00C3B012B23
:106860000CE08C2B65D005D8832B30D0862B40F0E4
:10687000BF8032E08D2B63D0933B022B00F2B880B7
:106880003FE0C82B00F083800FD8C12B6AD005D819
:10689000B52B60D0C02B40F0AB802BE0C32B6FD06A
:1068A00067D3C72B40F0A4801DE0D42B00F0848078
:1068B00005D8CC2B72D0D22B40F09A8075E0D62B25
:1068C00000F088807FD3FE2B40F0928089E000208A
:1068D000062103F0DDFF00F05EBD00200C2103F077
:1068E000D7FF00F058BD0D4B4920597A01F038FA16
:1068F00000F051BD094B4A20997A01F031FA00F0BD
:106900004ABD0020142103F0C3FF00F044BD00BFC6
:1069100044060020EC0A0020480B0020540B002005
:10692000BC06002050060020042103F0B1FF00F057
:1069300032BD4B20A149012201F094F900F02BBD9A
:1069400000201A2103F0A4FF00F025BD182103F058
:106950009FFF00F020BD58209949042201F082F9E0
:1069600000F019BD974B4820197A01F0F9F900F0B1
:1069700012BD40209349042201F074F900F00BBDD0
:1069800044209149042201F06DF900F004BD5F201C
:106990008E49012201F066F900F0FDBC4E208C49C1
:1069A000022201F05FF900F0F6BC50208949042270
:1069B00001F058F900F0EFBC54208749042201F09F
:1069C00051F900F0E8BC5E208449012201F04AF947
:1069D00000F0E1BC5C208249022201F043F900F0A2
:1069E000DABC4C207F49012201F03CF900F0D3BC15
:1069F0007D4B03221A7000F0CEBCFEF7D9FD00F0EB
:106A0000CABCFEF7EDFF00F0C6BCFFF7EBF900F0E3
:106A1000C2BC9378022B11D15378372B0AD8734913
:106A200003F5A77001EB83018000042201F01AF93D
:106A300000F0B1BC03232B7000F0ADBC04232B701D
:106A400000F0A9BC6A4B9A78022A12D15B78372BE6
:106A50000AD8664903F5A77001EB83018000023272
:106A600001F0C4F800F097BC5F4B03221A7000F0ED
:106A700092BC5D4B04221A7000F08DBCFFF7FCFA4B
:106A800000F089BCFFF7D8FB00F085BCFFF70CFCD9
:106A900000F081BC5278574B092A53D8DFE802F046
:106AA000050D151D26313941494C514A1968506868
:106AB000D27842EA0022521843E04D4A19685068E1
:106AC000D27842EA00228A1A3BE0494A19685068A3
:106AD000D27842EA00224A4333E0454A19685068B6
:106AE000D27842EA002291FBF2F22AE0404819688B
:106AF0004468C27842EA042291FBF2F002FB1012D1
:106B00001FE03B4A19685068D27842EA00220A40E6
:106B100017E0374A19685068D27842EA00220A43DF
:106B20000FE0334A19685068D27842EA00224A409E
:106B300007E01A68D24304E02D4A5168D27842EA4D
:106B400001221A602B4A2C4B12682AB91A6842F0AB
:106B500008021A6000F01FBC1A6822F008021A60CE
:106B600000F019BC224B234A5968DB78126843EACB
:106B700001239A4206DD204B1A6842F0040222F0FB
:106B800003020CE01C4B05D11A6822F0060242F009
:106B9000010204E01A6822F0070242F002021A60C1
:106BA000144A154B126822B91A6842F008021A609A
:106BB000F1E31A6822F008021A60ECE35F0B002090
:106BC0006C0B0020540B0020580B0020730B00208E
:106BD000620B0020640B0020680B0020720B002069
:106BE000700B0020600B0020BC060020CC060020AB
:106BF00044060020A40600204C06002053780C2BED
:106C000000F2C983DFE813F00D001B0029003700F4
:106C10004500530061006F007D008B009900A700C4
:106C2000B500944B1B6813F0080F00F0B483924B2F
:106C30005A68DB7843EA0222904B9A60ABE38D4BB3
:106C40001B6813F0080F40F0A6838B4B5A68DB7863
:106C500043EA0222894B9A609DE3864B1B6813F03E
:106C6000010F00F09883844B5A68DB7843EA0222D4
:106C7000824B9A608FE37F4B1B6813F0010F40F04B
:106C80008A837D4B5A68DB7843EA02227B4B9A6009
:106C900081E3784B1B6813F0040F00F07C83764B84
:106CA0005A68DB7843EA0222744B9A6073E3714BB3
:106CB0001B6813F0050F00F06E836F4B5A68DB788A
:106CC00043EA02226D4B9A6065E36A4B1B6813F03E
:106CD000020F00F06083684B5A68DB7843EA0222B7
:106CE000664B9A6057E3634B1B6813F0030F00F089
:106CF0005283614B5A68DB7843EA02225F4B9A6009
:106D000049E35C4B1B6813F0100F00F044835A4BAF
:106D10005A68DB7843EA0222584B9A603BE3554BB2
:106D20001B6813F0200F00F03683534B5A68DB7852
:106D300043EA0222514B9A602DE34E4B1B6813F03D
:106D4000400F00F028834C4B5A68DB7843EA02225C
:106D50004A4B9A601FE3474B1B6813F0800F00F00B
:106D60001A83454B5A68DB7843EA0222434B9A6008
:106D700011E3404B1B6813F4807F00F00C833E4B03
:106D80005A68DB7843EA02223C4B9A6003E33A4AB2
:106D90005168D27842EA01229A60FCE2374BDA6805
:106DA000072A00F2F88234499C684868C97841EAA9
:106DB0000020511C03EB8202C2F8F0409860D960B9
:106DC000E9E2DA682D4B002A00F0E582013A03EB94
:106DD0008201D1F8F010DA609960DCE253782E2B52
:106DE00003D8274A0121D154D5E2FF2B03D1234BED
:106DF00001225A74CFE203232B70CCE21E4B5B7846
:106E00002E2B03D81E4A0021D154C4E2FF2B03D1FC
:106E10001A4B00225A74BEE21A4B03221A70BAE2CD
:106E2000FFF760F9B7E2154B002283F8D120B2E2F8
:106E3000FEF734FBAFE2FEF7B7FCACE2FEF770FB07
:106E4000A9E20D4A104B52780A2A52D8DFE802F024
:106E5000060B20252B33393F45494C000B491A6856
:106E600009688A1803E0094A196812688A1A1A60C0
:106E70003FE000BF4C060020440600202C0200200A
:106E8000CC0B0020BC060020A4060020C406002075
:106E9000934A196812684A43E9E7914A19681268E7
:106EA00091FBF2F2E3E78E4A1968126891FBF2F067
:106EB00002FB1012DBE78A491A68096801EA02023C
:106EC000D5E787491A68096841EA0202CFE7844991
:106ED0001A68096881EA0202C9E7814B1A68D2433D
:106EE000C5E71A687E4BC2E77D4A186811681060D2
:106EF00019607C4A7C4B126822B91A6842F0080279
:106F00001A6048E21A6822F008021A6043E2754BE0
:106F100001F07F4118681B7841EA10215160D3705D
:106F2000FDF738FD37E26F4B01F07F4118681B78A1
:106F300041EA10215160D370FEF752FD2BE26B4BFA
:106F40005B78052B00F22782DFE803F003090F15B9
:106F50001B21654B1A6802F00F021A601BE2624B9C
:106F60001A6822F010021A6015E25F4B1A6822F0CC
:106F700020021A600FE25C4B1A6822F040021A608D
:106F800009E2594B1A6822F080021A6003E2564B5C
:106F90001A6822F480721A60FDE153782E2B04D80F
:106FA000534A02EB83035861F5E103232B70F2E1AE
:106FB0004F4BDFF830C1D3F810914E4993F82C2194
:106FC000D3F814A1CCF80090DFF814C1D3F81871ED
:106FD000D3F81C81D3F82061D3F82451D3F8284189
:106FE000CCF800A0885CDFF800C19F60CCF800807E
:106FF0001E74C3F8EC50C3F8E84008B101238B5469
:107000003B4B00229A74C6E193786BB9374B5B789F
:10701000142B05D8334A1168374A42F82310BAE1D5
:10702000364B03221A70B6E1344B04221A70B2E1D7
:1070300001F078FDAFE101F077FDACE101F076FD04
:10704000A9E101F075FDA6E101F074FDA3E101F0F5
:1070500073FDA0E101F072FD9DE101F071FD9AE187
:10706000234B002283F8D12095E1537813B1012BF3
:1070700010D104E01E4B012283F8D1208BE1B0F542
:10708000006F04D21A4A906082F8D13083E1042361
:107090002B7080E103232B707DE1154B022283F8D6
:1070A000D12078E1124B002199745974104A4FF0A5
:1070B000FF3402F1140040F821400E4800234354ED
:1070C00001312F29F2D1084913740B60054982F868
:1070D000D1300B60024993600B60D3605BE100BF6D
:1070E000C4060020A40600204C0600204406002010
:1070F0002C020020CC0B002050060020BC060020F3
:107100008D4B1B7D13F0020F0CD1B0F5006F06D232
:107110008A4B0422C3F8300183F8D1203BE10423D9
:107120002B7038E108232B7035E1844B002283F863
:10713000D12030E1804B01219A78814BB0F5006F6E
:107140001970804B1A7028D27B4B1C7D0C4024D1C7
:10715000694600F00DFF7B4B9DF800709DF80160C3
:107160009DF802509DF806C09DF805009DF804109A
:107170009DF803201C725F709E70DD7083F804C060
:1071800058719971DA7101236E4A985C117A013352
:107190004118082B1172F7D1FDE00123694A002143
:1071A00099540133082BF9D113781372F3E0537813
:1071B0008BB9614A01209178634A1468604A107063
:1071C000604A11700133E21812F8011C5D4A082B65
:1071D0009954F7D1DFE0012B40F0DD8014222A71B1
:1071E0000422EA717132AA716B71D4E0574B5B785B
:1071F000032B00F2D080DFE803F002101D224F4A7B
:10720000534BD2F8301192F8D1C0107C0A0A197190
:1072100083F807C098715A71BDE0484A4C4B916899
:1072200092F8D1C0107C0A0A197183F807C09871CE
:107230005A71B0E0474B1A68454B5A60ABE0464B79
:107240001A68434B5A60A6E0FEF7B0FBA3E0527801
:10725000424B02B101221A703C4B414AD878374B5D
:10726000107093F834113F4A002311703E4A137096
:107270003E4A13708FE0314B012283F835218AE0BA
:10728000FEF7DEFA87E0314B5B78032B4CD8DFE862
:1072900003F00C023C472D4B28495A68DB78D1F8A3
:1072A000381143EA022C00232BE0244BD3F8382179
:1072B000092A0CD82549501C4C68C97803EB820276
:1072C00041EA0421C2F83C11C3F8380163E0204BC5
:1072D00009221A705FE052F82340581C64450FD110
:1072E00002EB8002013904E052F8040C013342F849
:1072F000080C04328B42F7D3104BC3F838114AE024
:1073000003468B421A4AE6D345E00C4A0023C2F8F2
:107310003831174A0021D1500433282BF9D13AE0F3
:107320000B4B0A225A6036E0094B03221A7032E0F6
:10733000FFF70EF82FE000BF040000202C02002011
:10734000A8060020AC060020000000204406002013
:10735000BC060020A4060020C4060020D80A002095
:10736000F40A0020BA0B0020FB0B0020ED0A0020DD
:1073700068030020094B5A68DB7843EA022240F296
:10738000D2439A4207D1064B012283F8642102E0DE
:10739000044B02221A70BDE8FC8700BF440600209F
:1073A0002C020020BC06002073B5204B024640781A
:1073B0001F4D1870907800265870D078EC46987061
:1073C00010790C4698715079587192F806E095E85A
:1073D000030083F804E0D2798CE80300DA70154BDF
:1073E0001E70FEF7FFFF144B1B7873B96370237098
:1073F0002B78A3706B78E370EB792371AB796371B1
:107400006B79A3712B79E37108E0012B06D10B4B4B
:107410009B195B78A3550136082EF8D1044B6A46B8
:1074200092E8030083E803007CBD00BF440600200F
:10743000BC060020B6060020A8060020AC060020EE
:10744000F7B5114D114C6F684FF0000C07F07F47F6
:1074500047EA13276F600E4F6E4687F800C028700A
:107460006970AA7094E80300EB7086E80300FEF7E9
:10747000B9FF96E803006368227884E803000549B1
:1074800018460A70FEBD00BF44060020BC0600205E
:10749000B60600202C0200202DE9F04F804B93B05F
:1074A0001B781BB97F4B93F865316BB17E4B1B7812
:1074B000062B09D00A2B07D00F2B05D01F2B03D08A
:1074C000784B002283F83421764A92F83431032B2A
:1074D00025D192F8D040002C40F08680734B1B7869
:1074E00093B9734D734CA8786E78227863788619B7
:1074F000B618E279F618A379B6186279F6182379E6
:10750000B618F618F6B219E0012B40F09A806A4BD3
:10751000E05C013400F018FE092CF8D191E0042B56
:1075200027D1634D634CAB786E7818469E190136AF
:107530000023012222706360F6B2637000F004FE43
:10754000687800F001FE207800F0FEFD607800F021
:10755000FBFDE07900F0F8FDA07900F0F5FD607921
:1075600000F0F2FD207900F0EFFD304600F0ECFD78
:1075700067E0072B3CD192F8D030002B34D14B4A36
:10758000127822BB4A4A4B4B557896781C7893F870
:1075900001C0AF19D879E719997967445A79C719A1
:1075A0001B79CF19D719DF198DF838708DF8306035
:1075B0008DF831508DF832408DF833C08DF834009D
:1075C0008DF835108DF836208DF8373008E0012A17
:1075D00006D1394A995C0CAAD1540133092BF8D150
:1075E000364B1B786BB328E0324803F055FC28E09B
:1075F000082B26D12E4B0022597898782F4B45180E
:107600001C782C4B4FF0010C01355A608DF832C0BC
:107610008DF8332016468DF834208DF835208DF8FE
:1076200036208DF837208DF838505A7083F800C016
:107630008DF830008DF831101CB10CA8092101F033
:10764000E1F81F4B1B78002B6CD01E4B1B78032BD3
:1076500002D0072B61D139E0154C1B4DA07866781C
:107660002B7886190A36F61800F06EFD607800F067
:107670006BFD802000F068FD8A2000F065FD002091
:1076800000F062FD002000F05FFD002000F05CFDD6
:10769000F6B2287800F058FD304600F055FD3CE089
:1076A000B50600202C02002044060020A806002079
:1076B00004000020BC060020AC060020D00A0020F8
:1076C000FB0B0020BA0B0020ED0A00209E4B6FF050
:1076D0007F05597898789D4B00EB010C1A789C4BEC
:1076E0000CF10A0C1C78944400238DF826500A35BE
:1076F0008DF827508DF82A308DF82CC08DF8240095
:107700008DF825108DF828308DF829308DF82B2034
:107710001CB109A8092101F075F88E4A00231370E5
:107720008A4A13708C4B8D4893F8641100220270C2
:1077300083F8652183F8342111B10120FCF7F2FEB2
:10774000854B93F8352152B193F8D0200021D2F126
:10775000010238BF002283F8351183F8D0207E4C17
:1077600094F8D050002D73D10DF1470000F0BAFC11
:1077700000286DD000F0D2FC08B184F86651764B39
:107780009DF8470093F866114A1CD2B2C918092A1D
:1077900081F8680183F8662140F0EE806A4993F829
:1077A000682148784FF0000C904283F866C107D0FA
:1077B00091F82730002B00F0DF809A4240F0DC8007
:1077C000614B93F82730934203D1634B012283F836
:1077D000652100231A46604C04F5B471C95C01337D
:1077E0005218082BD2B2F6D194F8703193422DD1B1
:1077F0005B4B94F86D1194F86E2194F86F5194F8E6
:10780000696194F86AE194F86BC194F86C01DD70D9
:1078100059711A711E7083F801E083F802C09871E3
:1078200000F002FE4F4D94F8D1302860591E4E48AA
:107830000022C9B202700320012984F8340184F8BF
:10784000662160D9052B5ED001325DE004235EE045
:10785000414C94F8D03083B1414803F063FB60B1F0
:1078600000F0E2FD3F4994F8D13008603E495A1ECD
:1078700000200870D2B203213FE0374B93F8D0408C
:10788000002C47D1324B1B78002B43D00FA800F0BF
:10789000A3FF00283ED0234622460FA9C95C01332E
:1078A0005218082BD2B2F8D19DF844102A4C9142BC
:1078B0002DD12B4B9DF841109DF842209DF83D6045
:1078C0009DF83EE09DF83FC09DF840009DF8435074
:1078D00059711A711E70DD7083F801E083F802C0DF
:1078E000987100F0A1FD1F4994F8D13008601E493D
:1078F0005A1E00200870D2B20721012A84F83411E0
:1079000001D9052B1ED10022184B1A7034E084F8DF
:10791000343131E0104C94F8D130013BDBB2012B13
:107920002AD8A368B3F5006F22D2FCF76FFDF8B137
:10793000A3680B4918460133A36000F019FB092323
:1079400084F834310122DFE704000020ED0A002032
:10795000D00A0020FB0B00202C020020A8060020EB
:1079600044060020B40B0020B90B0020B60600200E
:10797000954B002283F8D120934C94F8D130042BFE
:1079800005D1924E327812F0800F00F0ED808E4BD0
:1079900093F834313BB1042B05D0082B03D0062BD0
:1079A00001D0FEF71FFD884C94F83431092B40F0CC
:1079B000B28000F039FDD4F8DC30854AC31A002BC0
:1079C0001268B8BF5B4293420AD9824B1A78012AE7
:1079D00001D101321A7000F027FD7B4BC3F8DC00A7
:1079E00000F022FD784BD3F8E020794B821A002A70
:1079F0005B68B8BF52429A420AD9764B5A78012A3C
:107A000001D101325A7000F00FFD6F4BC3F8E00056
:107A100000F00AFD6C4BD3F8E4206D4B821A002A6B
:107A20009B68B8BF52429A420AD96A4B9A78012A97
:107A300001D101329A7000F0F7FC634BC3F8E40007
:107A4000614A537C002B66D0937C002B63D19C460B
:107A5000614B92F82C011B68029007935F4BD2F8A0
:107A6000E8001B68039006935D4BD2F810811B68F9
:107A7000D2F814710593D2F8EC30D2F8184104937F
:107A8000D2F81C619368107CD2F82051D2F824B14E
:107A9000D2F8282101926246DFF83891194619F888
:107AA00002A0BAF1020F18D14E4951F82210B1F1DB
:107AB000FF3F0ED00546D0B202900398DDF810B01B
:107AC0000190059E069FDDF81C804FF0010C002000
:107AD00004E0002109F802101946234601322F2A3A
:107AE00002D01C460B46D7E7374AC2F8183110744B
:107AF000019B029882F812C0C2F81081C2F814717A
:107B00009160C2F81C61C2F82051C2F824B1C2F8D9
:107B1000283182F82C012C4B93F83421092A06D104
:107B200093F8D110022902D1033183F8D110264BEA
:107B3000D3F83811002944D0092A42D193F8D12032
:107B4000012A3ED19868002308E054F8234001330D
:107B5000A04203D1052382F8D13032E01A4A8B4289
:107B600002F59E74F1D32CE094F834314BB3042B1E
:107B700027D0082B25D0062B23D0F3787168D4F8B2
:107B80003001194D43EA0123B0F5006F6A706B6054
:107B900012D2314600F01CF93146D4F8300100F021
:107BA0003FF930B1D4F830310133C4F830316523B6
:107BB00000E007232B7004E007232B70002384F8D8
:107BC000D13013B0BDE8F08F2C0200204406002015
:107BD0007C0B0020CC0B0020A4060020C406002053
:107BE0004C06002040020020BC06002070B5044670
:107BF00000200E46154603210246FCF743FD0020F7
:107C0000C4F307210246FCF73DFD0020E1B2024625
:107C1000FCF738FD002407E0944214BF0022012243
:107C2000FCF730FD3055013400206A1EAC4201469D
:107C3000F2D370BD10B50446002003210246FCF7C4
:107C400021FD0020C4F307210246FCF71BFD0020A4
:107C5000E1B20246FCF716FD002001460122FCF7C6
:107C600011FD10BD2DE9F04104460F4616460020D7
:107C700006210122FCF706FD002005210246FCF743
:107C800001FD002001220146FCF7FCFC10F0020F70
:107C9000F2D0002002210246FCF7F4FC0020C4F3DD
:107CA00007210246FCF7EEFC0020E1B20246FCF799
:107CB000E9FC002543E0013414F03F08795D01D16F
:107CC000012204E0721E954214BF0022012200200E
:107CD000FCF7D8FCB8F1000F30D1731E9D422DD2B5
:107CE000002005210246FCF7CDFC002001220146C0
:107CF000FCF7C8FC10F00100F2D106210122FCF7CC
:107D0000C1FC002005210246FCF7BCFC002001223A
:107D10000146FCF7B7FC10F0020FF2D00020022160
:107D20000246FCF7AFFC0020C4F307210246FCF733
:107D3000A9FC0020E1B20246FCF7A4FC0135B542E3
:107D4000B9D3002005210246FCF79CFC002001224B
:107D50000146FCF797FC10F0010FF2D1BDE8F0816D
:107D600038B5012204460D4600200621FCF78AFCA6
:107D7000002005210246FCF785FC00200122014677
:107D8000FCF780FC10F0020FF2D000200221024626
:107D9000FCF778FC0020C4F307210246FCF772FCD4
:107DA0000020E1B20246FCF76DFC294600200122CA
:107DB000FCF768FC002005210246FCF763FC00206C
:107DC00001220146FCF75EFC10F0010FF2D138BD34
:107DD00038B50725454305F500650C462846097862
:107DE0000135FFF7BDFF284661780135FFF7B8FF81
:107DF0002846A1780135FFF7B3FF2846E178013521
:107E0000FFF7AEFF284621790135FFF7A9FF284685
:107E10006179FFF7A5FF681CA179FFF7A1FF38BDC5
:107E20002DE9F3470725454300200C460246032170
:107E3000FCF728FC05F500650020C5F30721024684
:107E4000FCF720FC0020E9B20246FCF71BFC0020F6
:107E500001460246FCF716FC824600200146024617
:107E6000FCF710FC8046002001460246FCF70AFCA5
:107E70000746002001460246FCF704FC814600202C
:107E800001460246FCF7FEFB06460020014602467C
:107E9000FCF7F8FB0546002001220146FCF7F2FB47
:107EA000237853451DD1637843451AD1A378BB424B
:107EB00017D1E37821798DF804608DF805508DF89D
:107EC0000600627943EA012343EA0243A079019A5A
:107ED00043EA006049EA0229814514BF00200120DD
:107EE00000E00020BDE8FC8738B54FF400640020B6
:107EF00006210122FCF7C6FB002005210246FCF703
:107F0000C1FB002001220146FCF7BCFB10F0020F70
:107F1000F2D0002002210246FCF7B4FB0020C4F39B
:107F200007210246FCF7AEFB0020E1B20246FCF757
:107F3000A9FB002500203F2D14BF0022012201468D
:107F40000135FCF79FFB402DF4D1002005210246AE
:107F5000FCF798FB002001220146FCF793FB10F090
:107F6000010FF2D14034B4F5804FC0D138BD00BF0D
:107F700038B50725454300200C4602460321FCF78F
:107F800081FB05F500650020C5F307210246FCF7DB
:107F900079FB0020E9B20246FCF774FB00200146A1
:107FA0000246FCF76FFB2070002001460246FCF7FA
:107FB00069FB6070002001460246FCF763FBA0707D
:107FC000002001460246FCF75DFBE0700020014600
:107FD0000246FCF757FB2071002001460246FCF7E1
:107FE00051FB6071002001460122FCF74BFBA071A0
:107FF00038BD00BF37B5002005210246FCF742FB23
:10800000002001220146FCF73DFB10F07104F2D183
:1080100000F00AFA054605E0FFF70CFE422814BFFF
:108020000024012400F000FA431B002BB8BF5B4280
:10803000B3F5FA6F40F2FF7002DA002CECD000E0EA
:108040001CB1234B1B78002B36D040F2FF7000216F
:10805000FFF786FEFFF748FF00201E494022FFF78A
:1080600001FE4FF480701C49B422FFF7FBFD402055
:108070001A492022FFF7F6FD002301934FF4C36451
:1080800001AD2046042204342946FFF7EBFDB4F588
:10809000FF6FF5D100230193A4F53074204604222C
:1080A00004342946FFF7DEFDB4F5C36FF6D140F284
:1080B000FF704221FFF754FE002040220549FFF7E0
:1080C00095FD402006492022FFF790FD3EBD00BFF0
:1080D000FC0A002004000020000001083000010814
:1080E000540B0020094B19685A68914201D10020B5
:1080F0000BE01A68D118097A013201701A601A6807
:10810000202A01D100221A6001207047A00300201C
:10811000014B9862704700BFA0030020034B1A7800
:10812000104612B100221A7001207047040C002082
:1081300008B5FCF74BF9034B00221A605A60FCF7B4
:1081400043F908BDA003002038B50B4B8446DC6A18
:108150001A6B0134202C08BF002494420AD0DD6A37
:108160000648ED1885F834C040F227710122DC6220
:1081700005F0D2FA38BD00BFA00300200044004043
:1081800038B50546002401E0FFF7DEFF2B5D013422
:108190001846002BF8D138BD2A4910B50B8813F0CA
:1081A000200F1CD0284BDB6813F0020F01D08B8806
:1081B00015E0264B5A6818680132202A08BF0022B1
:1081C000824205D05C688888E118C0B208725A60A3
:1081D0001F4B0A221A601D4B9A6A1E4B1A601948DF
:1081E000038813F0800F1BD01A4B1A68C2B9174BC3
:1081F000DC6A196B8C420FD0134902240C61196B95
:10820000CC1894F834C00131A0F804C01963196B7C
:10821000202905D11A6303E040F2277105F07CFAAA
:108220000848038813F0400F0BD040F2266105F098
:108230006BFB064B1A6BDB6A9A4202D1024B02229D
:108240005A6110BD0044004000080140A003002016
:10825000000C0020FC0B002030B5054687B05648C6
:1082600005F0A2FB4FF40030012104F0EBF90420EB
:10827000012104F0D9F90420002104F0F1F90820CB
:10828000002103F059FE06AC4FF0040324F8083D2A
:1082900003234A4821468DF8123015338DF81330E8
:1082A00003F0BAFD482345488DF8133021464FF0BE
:1082B0000803ADF8103003F0AFFD684605F0F6F99D
:1082C0000B2D25D8DFE805F02406090C0F12151830
:1082D0001B1E20224FF461531CE04FF4964319E01B
:1082E0004FF4E14316E04FF4164313E04FF46143BB
:1082F00010E04FF496330DE04FF4E1330AE04FF411
:10830000613307E02E4B05E02E4B03E02E4B01E0DE
:108310004FF416530093009B06A95B0841F8183DE3
:108320002548694605F0F8FA26230024012505A80A
:108330008DF8143007238DF815308DF816408DF820
:10834000175003F0D9FE1C4840F2FF3105F0B8FA8F
:1083500028212246184805F0DFF92A46164840F23F
:10836000277105F0D9F92A46134840F2266105F035
:10837000D3F92A46104840F2255105F0CDF922469E
:108380000D4840F2244105F0C7F922460A4840F65C
:10839000460105F0C1F92246074840F66A1105F08A
:1083A000BBF960212246044805F0B6F92946024887
:1083B00005F0A4F907B030BD0044004000080140BA
:1083C00090D0030020A1070040420F00704700BF7B
:1083D000104B1A787AB159680F4A01315960116807
:1083E0000E4B013111601A6812B11A68013A1A6015
:1083F0000022084B00E001221A70094B1A683AB1BA
:108400001A68013A1A601B6813B9064B01221A70E8
:10841000704700BFF4030020B8060020FC0B0020CA
:10842000000C0020040C0020014B5868704700BF6E
:10843000F403002008B5042004F026FB4FF4FA50A2
:1084400004F032FB012004F035FB04480321002234
:1084500003F020FF012004F043FB08BD9AC3020093
:1084600018B1082805D000200AE0064B188880B211
:1084700006E0044B588840F26B1380B25843001357
:10848000704700BFFC03002070B592B000244FF08D
:1084900003033A4811A98DF84630ADF844308DF801
:1084A000474003F0B9FC0120014604F0AFF8012178
:1084B0004FF4007004F0B8F8314803F0F7F8314B8E
:1084C00002260193304B2E48029380230693DB183B
:1084D000079303F540730893A3F5787301A90993F3
:1084E00003F5FF530A930394049605940B9403F049
:1084F0004DF92348012103F079F901254FF4602358
:1085000022480CA90E930C948DF834508DF83550F8
:108510000F948DF8406002F0FDFE1C4809212A46A8
:10852000032302F079FF032332461848082102F0A2
:1085300073FF224615484FF4FC6102F02FFF1348E9
:10854000294602F021FF1148294602F013FF0F4887
:1085500002F02EFF0D4802F031FF0028FAD10B483F
:1085600002F030FF094802F033FF0028FAD1074833
:10857000012102F031FF12B070BD00BF000C0140BC
:10858000080002404C240140FC030020002401406C
:10859000014B03221A60704700040020044A054B77
:1085A000927A0AB1052200E001221A60704700BFEA
:1085B000140C002000040020704700BF014B002273
:1085C0005A6070470004002008B5074B1A6892B241
:1085D00042F008021A601A6892B242F004021A606D
:1085E000FFF7D6FF08BD00BF405C004010B5064C49
:1085F0004FF6FB73226802EA03032360FFF7CEFF06
:108600004FF40643236010BD405C0040072818BFAC
:108610001F4B10B51E4C18BF18702378052B33D88C
:10862000DFE803F003060A0E1621FFF7DFFF2BE059
:10863000FFF7DCFF042328E002236370013324E00A
:108640006378013BDBB263706378FBB9042218E006
:10865000104B1A6892B242F010021A600523237080
:10866000DB18637012E06378013BDBB26370637800
:1086700063B9084A4FF6EF73116801EA0303136008
:108680000622034B1A7001E00623237010BD00BFC1
:10869000780C0020405C0040034B9B7A13B1034BE5
:1086A00005221A60704700BF140C0020000400204F
:1086B000014B04221A60704700040020034B1A7A11
:1086C000202A01D100221A72704700BF0004002046
:1086D000704700BF212808B508D1124B1B681B78D2
:1086E00003F07F03212B1AD10F4B0EE0202816D167
:1086F0000C4B0E4A1B681B7810720D4A03F07F0367
:10870000212B0CBF134600234BB1064A4FF000014A
:1087100012680020518293619847002000E00220F7
:1087200008BD00BF740C0020698700080004002009
:1087300085870008074B1B681B7803F07F03212BFC
:1087400005D1022801D0222801D1002000E002201A
:10875000704700BF740C002019B9012801D80846E1
:1087600000E00220704700BF28B9044B4FF0080218
:108770001B681A8200E00248704700BF740C00209A
:108780004400002028B9044B4FF008021B681A82ED
:1087900000E00248704700BF740C00204400002035
:1087A0000B4B10B5DA6882B11B68052B01D0002293
:1087B0000BE0002303E00749595CC154013304492D
:1087C000CC68A342F7D30023CB60104610BD00BF96
:1087D000000400207C0C0020084BDB68082B01D82B
:1087E00000200AE00023064A9A5CC2540133092B98
:1087F000F9D1024B0022DA6001207047000400200A
:108800007C0C002010B5074C0B468AB2C021636077
:1088100005F0A6FE0120A18806F0B0F8012005F0C1
:108820007BFF10BD0004002007B5142200238DF843
:10883000042001A801228DF806308DF807208DF85C
:10884000053003F059FC0EBD07B5142200238DF846
:10885000042001A801228DF806308DF807208DF83C
:10886000053003F049FC0EBD08B5064B1B68DB78EC
:10887000042B01D9002004E0034901EBC30105F0FA
:1088800017FA08BD740C00204C00002008B50249FE
:1088900005F00EFA08BD00BF6C00002008B50249C3
:1088A00005F006FA08BD00BF74000020334B10B578
:1088B0001B686FF03F0200245A72DC729C722046E3
:1088C00005F0A2FE20464FF4007105F0BBFE10211A
:1088D000204605F0CDFE4021204606F023F88021F9
:1088E000204606F00FF8204605F04CFF244B2046AA
:1088F00093F8641006F064F8204605F01BFF012091
:10890000214605F09FFE0120C02105F0FBFF01205C
:10891000202105F0ADFE0120214605F0C1FE022018
:108920004FF4C06105F08EFE02204FF4807105F017
:10893000E9FF0220214605F0B3FE0220202105F0C8
:1089400097FE0320214605F07DFE03204FF4887139
:1089500005F0E8FF0320402106F032F803204FF431
:10896000405105F09DFE2146032005F081FE204682
:1089700005F0ACF9034B01221A6010BD740C002005
:10898000440000200004002008B5174B174A19685E
:1089900089B2118016491288098801EA020212F48C
:1089A000806F05D04FF6FF321A60124BDB6B984791
:1089B0000E4B1A880E4B1B8803EA020212F4007F4A
:1089C00008D009490C4A4FF6FF500860117C01316C
:1089D000C9B21174054A1288134013F4004F01D034
:1089E00005F0FAFC08BD00BF445C00400A0C002002
:1089F000BC0C0020440000200004002010B503201F
:108A000006F00EF8064C034602464FF488710548FE
:108A1000E36005F0BDFD032005F08CFE10BD00BF36
:108A2000000400207C0C002008B520B1044801217E
:108A300003F058FA03E00248012103F055FA08BD9B
:108A40000008014038B5064D01232B60054B00247A
:108A500020461C60FFF7E8FF03232B60204638BD4B
:108A6000405C0040445C004008B5FFF7EBFF08BDE8
:108A700008B50120FFF7D8FF064B01211960064910
:108A80004FF4E0520A8005490020186008601A601F
:108A900008BD00BF405C0040BC0C0020445C0040AE
:108AA000084B10B51B6800249C72FFF7E1FF064AD3
:108AB0004FF406431460043A1360044A1460044AF5
:108AC000138010BD740C0020445C004000040020A2
:108AD000BC0C0020012008B503F01CFD4FF4000081
:108AE000012103F0AFFD08BD07B5FFF7F3FFFFF766
:108AF000ABFE05F013FC0420012103F095FD0323D8
:108B00008DF806300D338DF8073004484FF001031F
:108B100001A9ADF8043003F07FF90EBD0008014053
:108B2000704700BF704700BF704700BF704700BF6D
:108B3000704700BF704700BF704700BF704700BF5D
:108B4000704700BF10B5FFF76FFC074C2368C31ACE
:108B5000B3F5FA7F07D9054BDA6882F40072DA6060
:108B6000FFF762FC206010BDC00C0020000C01402B
:108B7000024B03EBC003D879704700BF14040020F8
:108B8000024B03EBC0035879704700BF1404002068
:108B9000024B03EBC0039879704700BF1404002018
:108BA000024B0B2202FB0033187A7047140400209A
:108BB000024B0B2202FB0033587A7047140400204A
:108BC000024B0B2202FB0033D87A704714040020BA
:108BD000024B0B2202FB0033987A704714040020EA
:108BE000024B0B2202FB0033187B70471404002059
:108BF000024B0B2202FB0033587B70471404002009
:108C0000024B0B2202FB0033987B704714040020B8
:108C1000024B0B2202FB0033187C70471404002027
:108C2000024B0B2202FB0033587C704714040020D7
:108C3000024B0B2202FB0033987C70471404002087
:108C4000024B052202FB0033187D704714040020FC
:108C5000024B052202FB0033587D704714040020AC
:108C6000024B052202FB0033987D7047140400205C
:108C7000024B052202FB0033D87D7047140400200C
:108C8000024B052202FB0033187E704714040020BB
:108C9000024B032202FB0033187F704714040020AC
:108CA000034B032202FB003393F91D00704700BF02
:108CB00014040020024B032202FB0033987F70470C
:108CC00014040020024B03EBC00393F8200070470C
:108CD00014040020024B03EBC00393F821007047FB
:108CE00014040020024B03EBC00393F822007047EA
:108CF00014040020024B03EBC00393F823007047D9
:108D000014040020024B03EBC00393F824007047C7
:108D100014040020024B03EBC00393F825007047B6
:108D200014040020024B03EBC00393F826007047A5
:108D300014040020024B03EBC00393F82700704794
:108D40001404002006281AD8DFE800F004070A0DF2
:108D5000101316000A4B9B6A10E0094BDB6A0DE00A
:108D6000074B1B6B0AE0064B5B6B07E0044B9B6BEE
:108D700004E0034BDB6B01E0014BDB7B0B607047D6
:108D80001404002070B5C0F30741054600220120FD
:108D9000FBF778FC0A4C0602C5F3072100220120EC
:108DA000A662FBF76FFC064301203602E9B20246D9
:108DB000A662FBF767FC06433609A66270BD00BFDA
:108DC000140400202D4B032202FB003310B51C338A
:108DD00093F901203F2A01DD3F225A70274B0322DD
:108DE00002FB00331C3393F9012012F13F0FBCBF8B
:108DF0006FF03E025A70214B032202FB00331C33FA
:108E00009A781F2A01D91F229A701C4B032202FB59
:108E100000324FF440211964127F012A04BF4FF43D
:108E200050221A64154B03EBC00292F827203AB97E
:108E3000033202FB0032527F196C02F07F020BE01A
:108E4000032101FB003191F81DC002F003020CF078
:108E50007C0C196C4CEA0202084C41EA02221A64AA
:108E6000032303FB0040236C827F42EA030318467E
:108E70002364FFF787FF236CA36310BD1404002055
:108E800008B5044B032202FB00339977FFF79AFFE2
:108E900008BD00BF1404002008B5044B032202FBE8
:108EA00000335977FFF78EFF08BD00BF1404002080
:108EB00008B5044B032202FB00331977FFF782FF4A
:108EC00008BD00BF14040020264B052210B502FB8C
:108ED00000331A7D012A01D901221A75214B05227E
:108EE00002FB003314335A78032A01D903225A7043
:108EF0001C4B052202FB003314339A780F2A01D948
:108F00000F229A70174B052202FB00331433DA78D4
:108F1000032A01D90322DA70124B052202FB003327
:108F200014331A790F2A01D90F221A710D4C052317
:108F300003FB004000F114021379017D43F4202368
:108F4000507843EAC133917843EA4033D27843EA18
:108F5000012343EA421318462364FFF713FF236CEF
:108F6000636310BD1404002008B5044B052202FB06
:108F700000331976FFF7A8FF08BD00BF14040020D6
:108F800008B5044B052202FB0033D975FFF79CFF9F
:108F900008BD00BF1404002008B5044B052202FBE5
:108FA00000339975FFF790FF08BD00BF140400203F
:108FB00008B5044B052202FB00335975FFF784FF07
:108FC00008BD00BF1404002008B5044B052202FBB5
:108FD00000331975FFF778FF08BD00BF14040020A7
:108FE000514B0B2210B502FB00331A7A032A01D928
:108FF00003221A724C4B0B2202FB003308339A787F
:10900000032A01D903229A70474B0B2202FB00333B
:1090100008331A790F2A01D90F221A71424B0B22F9
:1090200002FB003308335A79072A01D907225A7103
:109030003D4B0B2202FB003308339A790F2A01D9EA
:109040000F229A71384B0B2202FB003310335A78EF
:109050000F2A01D90F225A70334B0B2202FB003327
:1090600010339A780F2A01D90F229A702E4B0B22B7
:1090700002FB0032117AC90341F400241C64527AC5
:1090800012B141F404211964274B0B2101FB00317B
:10909000C97A19B1196C41F400511964224B8AB98B
:1090A0000B3202FB0032083292F804C091784FEA8A
:1090B000CC1C1C6C4CEAC12C51794CEA040242EAEB
:1090C00001121DE00B2202FB0032127C1AB11A6C55
:1090D00042F480521A64144B0B2101FB0031103111
:1090E00091F801E01A6C897842EACE1201F0070C7F
:1090F00042EA0C1211F0080F1A6402D042F4006226
:109100001A64094B0B2202FB00300830C27922B9E5
:1091100081791A6C41EA02021A64034C206CFFF751
:1091200031FE236C236310BD1404002008B5064BE8
:109130000B2202FB00330833DA791AB10022DA710C
:10914000FFF74EFF08BD00BF1404002008B5064B12
:109150000B2202FB00330833DA791AB90132DA71D3
:10916000FFF73EFF08BD00BF1404002008B5044B04
:109170000B2202FB00339974FFF732FF08BD00BFDA
:109180001404002008B5044B0B2202FB0033597471
:10919000FFF726FF08BD00BF1404002008B5044BEC
:1091A0000B2202FB00331974FFF71AFF08BD00BF42
:1091B0001404002008B5044B0B2202FB0033997302
:1091C000FFF70EFF08BD00BF1404002008B5044BD4
:1091D0000B2202FB00335973FFF702FF08BD00BFEB
:1091E0001404002008B5044B0B2202FB0033197352
:1091F000FFF7F6FE08BD00BF1404002008B5044BBD
:109200000B2202FB00339972FFF7EAFE08BD00BF94
:109210001404002008B5044B0B2202FB0033D97262
:10922000FFF7DEFE08BD00BF1404002008B5044BA4
:109230000B2202FB00335972FFF7D2FE08BD00BFBC
:109240001404002008B5044B0B2202FB00331972F2
:10925000FFF7C6FE08BD00BF1404002010B5254B63
:109260004FF460221A6403EBC00292F8272012B177
:109270004FF470221A641F4B03EBC00292F82110C6
:1092800092F820C01C6C090341EA8C312143196417
:1092900092F82220012A04BF41F480611964154B21
:1092A00003EBC00191F823C01A6C42EA0C221A6445
:1092B00091F82410012904BF42F080021A640D4B7A
:1092C00003EBC00292F82520012A03D11A6C42F068
:1092D00040021A64074C04EBC00090F82620236C6F
:1092E00043EA021318462364FFF74CFD236CE36343
:1092F00010BD00BF1404002008B5044B03EBC003ED
:1093000083F82610FFF7AAFF08BD00BF1404002051
:1093100070B50F4B064603EBC00393F82650032DA0
:1093200002D00321FFF7E8FF3046FFF797FF084B15
:109330009C6A14F4002F1CBF6FEA04346FEA1434E3
:10934000032D03D030462946FFF7D6FF204670BDD7
:109350001404002008B5044B03EBC00383F8251068
:10936000FFF77CFF08BD00BF1404002008B5044BC4
:1093700003EBC00383F82410FFF770FF08BD00BFA4
:109380001404002008B5044B03EBC00383F823103A
:10939000FFF764FF08BD00BF1404002008B5044BAC
:1093A00003EBC00383F82210FFF758FF08BD00BF8E
:1093B0001404002008B5044B03EBC00383F821100C
:1093C000FFF74CFF08BD00BF1404002008B5044B94
:1093D00003EBC00383F82010FFF740FF08BD00BF78
:1093E00014040020064B10B503EBC003044683F8B9
:1093F0002710FFF733FF2046FFF7E4FC10BD00BF46
:109400001404002010B5144B00221A6403EBC002B0
:10941000527912B14FF400721A640F4B03EBC00281
:1094200092791AB11A6C42F480721A640A4B03EBF7
:10943000C003DA790F2A01D90F22DA71064C04EB46
:10944000C000C279236C42EA030318462364FFF785
:1094500099FC236CE36210BD1404002070B5084D24
:109460009DF810E09DF8146005EBC0042671627051
:10947000A37084F803E005F83010FFF7C3FF70BD58
:109480001404002008B5034B03EBC0039971FFF7E8
:10949000B9FF08BD1404002008B5054B03EBC00359
:1094A000597109B10422DA71FFF7ACFF08BD00BFA2
:1094B0001404002008B5054B042903EBC003D9713F
:1094C00001D000225A71FFF79DFF08BD140400204F
:1094D0002DE9F047344D0446401990F844000E46FB
:1094E00017469846DDF82090DDF824A004281FD800
:1094F000DFE800F003090F151B002046FFF770FDA1
:109500006519012316E02046FFF7A8FE651902231E
:1095100010E02046FFF7D8FC651903230AE0204637
:10952000FFF750FC6519042304E02046FFF76AFFAB
:109530006519002385F844301B4B03EBC40494F8F1
:109540002620012A0DD002D3022A23D111E016B120
:109550009B6A9B0C3370EFB1134B9B6A9B0A3B7069
:1095600018E0B8F1000F15D09B6A9B0AC8F80030CC
:1095700010E0B8F1000F04D09B6ADB0B5B01C8F868
:109580000030B9F1000F05D0074B9B6AC3F3842369
:1095900089F80030BAF1000F03D0034B9B6A8AF8B8
:1095A0000030BDE8F08700BF14040020214B10B547
:1095B000032200244FF0050C02214FF0010E83F826
:1095C00025E0197383F80EC09A745C7483F81CE06C
:1095D00083F81DC083F81EC083F8202083F8212063
:1095E00083F8224083F8234083F8244083F8261030
:1095F00083F827401C755C759C75DC751C765C7166
:109600009C71DC7119725C72DC729C725A73DC732F
:109610001C742046FFF758FC2046FFF7D3FB20467A
:10962000FFF71CFE2046FFF7EDFE2046FFF7D8FCB3
:1096300010BD00BF1404002008B5044A0023917A2D
:10964000034A18461370FAF775FF08BD540B002043
:10965000BC0B0020F0B5804B85B01A7822B90132DE
:109660001A706FF000425A607B4B1C7A5CB9E0B212
:10967000FAF7FCFE784B03F10C0210550134082C6C
:10968000F5D101221A7227240025E8B2FAF7EEFE7E
:10969000724A535D834219D0714B291D53F8213012
:1096A0005055022B05D0032B0AD0012B0ED168B1E7
:1096B00006E058B96B4A115D012907D1135505E041
:1096C000684B1A5D012A01D101321A550135013466
:1096D000082DDAD1644EF36993B1644C25787DB9D5
:1096E000FEF7A2FE624AF3691268821A002AB8BF26
:1096F00052429A4204D9284601F0B2F9012323705C
:10970000594E336A93B15B4C25787DB9FEF78CFED8
:10971000594A336A1268821A002AB8BF52429A42E2
:1097200004D9284601F09CF9012323704A4D534C7B
:109730002A7D930004EBC3010E7B002E00F02981EB
:109740004F48504F504E0021C318BF18B61810464E
:109750000A4600970196FFF7BBFE2B7D04EB4314EE
:10976000227B013A042A00F20581DFE812F00500AD
:109770004E00D3004E00D300444A374D926812F495
:10978000004F1BD15D192A7E022A04D1404AD25CC7
:10979000002A00F0EF80394A2F4C02EB43121846A2
:1097A000517AFAF7C7FE207DFFF7C0FC237D384AC7
:1097B00000211C19D15402232376DBE05D192A7E97
:1097C000012A04D1324AD25C002A00F0D3802B4C0B
:1097D000184604EB4313997AFAF7ACFE1E4B187D3A
:1097E00004EB4014A37A13B9FFF7B0FC04E0284B54
:1097F0001B5C0BB1FFF79AFC174A2549137D00202B
:109800009A18C85401231376B4E01F4A124DD25659
:10981000002A3FDB5D192A7E022A02D11C4AD25C53
:109820008AB1164A0C4C02EB43121846517AFAF7E9
:1098300081FE207DFFF77AFC237D154A00211C194B
:10984000D15402232376044C257DFEF7EDFD04EB75
:109850008504606056E000BF5C04002068040020BE
:109860007C0B0020CC0B002004000020B90B002052
:10987000B40B0020D10A0020AC0B0020540B0020B8
:10988000F80A0020DC0A00204C0B002000080140F0
:10989000B80B00205B191B7E012B11D0FEF7C4FD15
:1098A0002B7D894A05EB830502EB43139B8B0A2230
:1098B00053436A68821A002AB8BF52429A4204DCB3
:1098C000824B834A1B7DD35CE3B1804D7E4C287D67
:1098D00004EB4013997AFAF72DFE287D04EB40142F
:1098E000A37A13B9FFF732FC04E0794B1B5C0BB190
:1098F000FFF71CFC754A7649137D00209A18C8545E
:1099000001231376714B1A7D6F4B03EB42131B7BC4
:10991000042B20E06D4A9A18127E022A02D16C4A6A
:10992000D25C8AB1684A694C02EB43121846517AFC
:10993000FAF700FE207DFFF7F9FB237D644A002142
:109940001C19D15402232376604B1A7D5E4B03EB26
:1099500042131B7B052B0DD15E4B9B6813F4004F0C
:1099600004D15D4B4FF480625A6103E05A4B4FF4CF
:1099700080621A61FEF758FD544CE369C31A002B4C
:10998000B8BF5B420A2B40F3AD82FEF74DFDE061AC
:10999000A8E2FEF749FDEB69C31A002BB8BF5B4292
:1099A0000A2B40F39F82297D3046490141F00A018C
:1099B00001F0EA0100F016FF0446287D01F074F87A
:1099C0002B7D0C20584345494218157A0DB1455856
:1099D00000E05568424AD25C032A00F2E780DFE8E3
:1099E00002F002831C4B002C00F0E080364A374D19
:1099F00002EB4311C97F3A4E29B11846FAF79AFD96
:109A00002B7D032207E002EB43121846517AFAF746
:109A100091FD2B7D0222F254C8E04CB95B0143F06A
:109A2000080101F0E801204600F0DCFE002865D0C6
:109A3000264E254B307D03EB4013D97F002900F0E3
:109A4000AE80002D84EAE472B8BF6D42A2EBE472EE
:109A5000AA4202D0002C40F09C80224B53F83010D8
:109A60008A4280F09C8003EBC0031979FAF762FD0B
:109A7000164B01211B7D90E0002D84EAE471B8BFF4
:109A80006D42A1EBE471A94202D0002C40F0878026
:109A9000144A0E4D52F83300114E814208D202EBA7
:109AA000C30218461179FAF745FD2B7D012208E023
:109AB000054A184602EB4313597AFAF73BFD2B7D12
:109AC0000222F2546BE000BF540B00205C04002023
:109AD000B80B002000080140000C0140000B0020E2
:109AE000BC0B0020E00A002044BB5B0143F00801EE
:109AF00001F0E801204600F075FEF8B9FEF794FC8D
:109B00001F4D204A2B7D4FF00A0E02EB4311B1F896
:109B10001CC099004E1976680EFB0CFC861B002EAB
:109B2000B8BF7642664541DD02EBC1021846917A24
:109B3000FAF700FD2B7D144AD45437E0104E114A39
:109B4000337D02EB4312D17F49B3002D84EAE472E6
:109B5000B8BF6D42A2EBE472AA4200D0C4B90B496F
:109B600051F833108A421AD3064A184602EB4313BF
:109B7000597AFAF7DFFC024B02211B7D0DE000BF92
:109B80005C040020540B0020BC0B0020E00A0020E5
:109B90001846FAF7CFFC337D03219D4AD1549D4DE1
:109BA0002E7DFEF741FC05EB86056860994D9A4FC6
:109BB0002B7D9A4E1846F618FF18994B002103EB9F
:109BC00080030A4601960097964EFFF781FC287D98
:109BD00006EB40139B6943B3FAF7ECFB28B3287DEF
:109BE00084EAE47206EB40139B69A2EBE4729A42AA
:109BF0001BD900F035FF2A7D8B4906EB42139B7F72
:109C00000120885443B1B27F9A4205D1013800F057
:109C100027FF002000F078F97E4B844A1B7D0F332C
:109C2000D15C012901D10131D1547A4D2B7D022B18
:109C300025D8002000F0B2FC95F8203010F0010F7C
:109C400003F0F80385F820301CBF43F0010385F8CA
:109C5000203010F0040F8DF80C0006D06D4B93F8F7
:109C6000202042F0020283F8202010F0100F06D0CE
:109C7000684B93F8202042F0040283F820206C4ABD
:109C8000137853B1634991F820100B4205D169490B
:109C900069480978037001B91170674B1B784BB1A3
:109CA0005C4A92F8202003EA02029A4202D1634BF6
:109CB00001221A70574B93F8202012F0010F0AD09E
:109CC00093F8213013F0010F05D1584BDA78012AAF
:109CD00001D10132DA704F4B93F8202012F0020FBD
:109CE0000AD093F8213013F0020F05D14F4B1A79A7
:109CF000012A01D101321A71464B93F8202012F04B
:109D0000040F0AD093F8213013F0040F05D1474B0C
:109D10005A79012A01D101325A713E4D03222B7D1D
:109D200004A8B3FBF2F2821812F9042C95F8201063
:109D3000002A85F821104ADA5B0143F01601002061
:109D400001F0F60102AA00F065FD9DF80A3013F05B
:109D5000400F08D02A7D354952001B32885C01280B
:109D600001D10130885413F0800F0AD029492F4ABD
:109D7000097D0E3112F81100012802D1013002F8DC
:109D8000110013F0100F09D0224A2849127D520009
:109D90001B32885C012801D10130885413F0200F58
:109DA0000AD01C4A214B127D0E3213F812100129E1
:109DB00002D1013103F81210164B0020197D02AABE
:109DC000490141F0160101F0F60100F0BFFE54B95F
:109DD000104B2046197D490141F0080101F0E801CE
:109DE00000F000FD28B10B4D154B2E7D9B5D002B27
:109DF00044D0084B0B4A1B7D02EB4312D2891AB99F
:109E00000F4AD35C002B3ED0FEF70EFB014D19E04C
:109E1000BC0B00205C040020DC0A00204C0B00205E
:109E2000F80A0020540B0020480B0020CC0B002027
:109E3000F40A0020D80A0020ED0A0020FB0B0020C5
:109E4000C40B002028492B7D4FF00A0C9A0001EB2F
:109E5000C201C9895219526A0CFB01F1821A002A07
:109E6000B8BF52428A420EDD204EF25C5AB9184603
:109E7000FFF76CF92B7D0122F25404E0FEF7D4FACF
:109E800005EB860568621A4E1A4D307D002C55F898
:109E90003030B8BF64429C420AD2FEF7F1FE337DF7
:109EA00005EBC3056A7982420DD11846002108E00E
:109EB000FEF7E6FE337D05EBC3056979884202D0E3
:109EC0001846FFF751F80A4C207D00F02BF8237D4F
:109ED0000133DBB223750BB100232375FEF7A4FA1F
:109EE000034BD86105B0F0BD540B0020C80B002017
:109EF0005C040020E00A0020024B1A5C0AB901321F
:109F00001A54704784040020024B1A5C0AB10F22D5
:109F10001A54704784040020014B185C704700BF3E
:109F2000840400202DE9F3474501EDB2044645F0D5
:109F30007C01002001AA00F06DFC4FEA440A0227D0
:109F4000012307FA0AF703FA0AF3B64A9DF8061046
:109F500002EB4412127A0B400F4012F0800F02F015
:109F60007F0804D0B04A966886F0200601E0AE4A29
:109F7000966808F1FF32C6F34016072A00F2D9822C
:109F8000DFE812F0080008000800080074017401FE
:109F900074017401A54A125D013A0E2A00F2C982C9
:109FA000DFE812F00F003D00550064007D008500E1
:109FB0009400A900D9001C012101C7024A015401E3
:109FC000AE0201AA45F014010020984E00F022FCD8
:109FD0009DF8053045F0060506EB84077B602946B1
:109FE000002000F0FFFB0222B8602146002000F0B4
:109FF00099FBA8F102080020294640F2FF7200F008
:10A00000FDFC5FFA88F800200322214600F064FB83
:10A01000B8F1010F40F2C6810423335589E2834E23
:10A02000002006EB84035A68214602F004028242B3
:10A0300014BF0522012200F04FFB7A4B6201D25877
:10A0400045F00801002000F0D9FC0323E5E7002BD0
:10A0500000F06F8245F00201002000F089FB734B95
:10A0600004221A55724B43F8240062E26F4E00201E
:10A0700006EB84035A68214602F00402824214BFB0
:10A080000622022200F028FB664B6201D25845F0FE
:10A0900008015242002000F0B1FC0523BDE7002F6B
:10A0A00000F04782204600F0DBFC062234E200206C
:10A0B0002146032200F010FB5A4B45F0080103EB48
:10A0C00044135A68002000F099FC72E1002F40F020
:10A0D000308245F00805384629463A4600F08EFCA5
:10A0E000504B384603EB44135A682946524200F05D
:10A0F00085FC082210E2002F00F01B8245F00201CF
:10A10000002000F035FB06460020024645F008011D
:10A1100000F074FC464B002053F824702146BF1B0E
:10A1200043F82470032200F0D7FA3E4B6701FB1876
:10A130005A6845F00601002000F060FC07F0E001DD
:10A140003246002000F0C6FB00200246214600F007
:10A15000E9FA0922E0E1002000F020FA40FA0AF0D2
:10A1600010F0010F00F0E58145F0020631460020B5
:10A1700000F0FEFA2F4B45F0080543F824000020BC
:10A180000246294600F03AFC00200222214600F057
:10A19000C9FA00203146024600F09CFB670100200E
:10A1A000A8F1030807F0E00102465FFA88F800F022
:10A1B00091FBB8F1010F1D4E0ED80020214602225E
:10A1C00000F0B0FA174B2946FF187A680020524277
:10A1D00000F014FC0A2320E70E231EE7002F00F0F6
:10A1E000A8810B2298E1002F40F0A38145F00201E5
:10A1F000384600F0BDFA45F0080106463A463846B2
:10A2000000F0FCFB6101022296FBF2F201F0E0019A
:10A21000384600F05FFB3A463846214600F082FAA5
:10A220000D2279E1540B0020000C01408404002031
:10A23000D40A0020780B0020002000F0AFF940FA8B
:10A240000AF010F0010F00F0748164E1A94E45F0AE
:10A25000060106EB84050020AA6800F0CFFB2A79EE
:10A260000020214600F038FA0023D6E6A14A125D0C
:10A27000013A0E2A00F25D81DFE812F00F0035008E
:10A28000570067008A005B019D005B015B01D30002
:10A29000E200B6000F015101420145F0140101AA8C
:10A2A0000020944E00F0B6FA9DF8057006EB84038A
:10A2B000002002225F60214600F034FA002045F0C1
:10A2C000060140F2FF7200F099FB002003222146B4
:10A2D00000F002FAB8F1060F03D0B8F1080F7FF4CE
:10A2E0009BAE022218E1B8F1060F0CD1814B002081
:10A2F00003EB84035A68214602F00402824214BF31
:10A300000522012205E0B8F1080F04D10020214602
:10A31000032200F0E1F9784B6201D25845F00801C0
:10A32000002000F06BFB0322F6E0A8F10502D2B298
:10A33000012A05D823B1B8F1060F6E4E34D16BE671
:10A34000002E00F0F6800C22E6E0B8F1050F0CD1EB
:10A35000684B002003EB84035A68214602F0040294
:10A36000824214BF0622022205E0B8F1070F04D191
:10A3700000202146032200F0AFF95F4B6201D25862
:10A3800045F008015242002000F038FB0522C3E0EE
:10A39000A8F10503DBB2012B08D83FB1B8F1050FD6
:10A3A000544E01D1022338E60F2336E6002E00F08A
:10A3B000C0800722B0E0002E40F0BB804D4F3046F9
:10A3C00007EB84035A68214602F00402002A14BFF6
:10A3D0000522012200F080F9474B304603EB44137D
:10A3E00045F008015A6818E0002E40F0A280414F65
:10A3F000304607EB84035A68214602F00402002A23
:10A4000014BF0622022200F067F93B4B304603EBF3
:10A4100044135A6845F00801524200F0EFFA0A234B
:10A4200039E0002E00F0858045F00201002000F0A8
:10A430009FF9304B0B2103EB84021955D06078E073
:10A44000002E76D145F00201304600F091F92A4BFA
:10A450004FEA44184FEA840A08EB0302254F03EB46
:10A46000CA03814645F00601526830465E7300F02B
:10A4700031FA0AEB0703DB6808F0E0019944022394
:10A4800099FBF3F2304600F025FA30462146324679
:10A4900000F048F90D233B554BE0002000F07EF81A
:10A4A00040FA0AF010F0010F43D0124B0E2245F093
:10A4B00002061A553146002000F05AF90F4B45F0BC
:10A4C000080143F824000020024600F097FA2146D4
:10A4D0000020022200F026F900203146024600F05A
:10A4E000F9F96101002001F0E001024600F0F2F903
:10A4F0001FE000BF84040020540B0020780B0020D4
:10A5000000202146022200F00DF9002045F008014C
:10A51000024600F073FA0E22074B1A5509E0064D69
:10A52000002005EB84031A79214600F0D5F80023BA
:10A530002B55BDE8FC8700BF84040020000000000C
:10A54000154B10B503EB0012926891420EDD8A1A8A
:10A55000C2F18074A2424FEA001C03DC63445C68D1
:10A5600012190EE063445A68141B0FE00FDA521AF6
:10A57000C2F18074A2424FEA001C04DC63445C68B0
:10A58000A21A5A6003E063445A68A4185C60024B44
:10A5900003EB0010816010BDC40C0020012108B540
:10A5A00002200A46FAF76EF808BD00BFF8B5137826
:10A5B000144613F0600F06460D4627D1414A127B20
:10A5C00022BB13F0010F21D15F2B1FD83E4A127816
:10A5D000E2B913F09F0301D0082B17D13B4F387815
:10A5E00060B9384BD97F19B1F9F7A4FF032304E010
:10A5F0000846597AF9F79EFF02233B70344F3B78A7
:10A6000023B10020FEF792FD00233B700022217849
:10A610000220FAF737F82870002261780220FAF752
:10A6200031F868700022A1780220FAF72BF8A870A0
:10A6300001220220E178FAF725F8E870237813F078
:10A64000010F3ED15F2B3CD803F01E02082A04D034
:10A65000142A2CD0062A34D11BE0242171435B0933
:10A660000C2000FB0313A57894F803C0194A4CEAA8
:10A6700005259D50A37813F0080F22D0267876097F
:10A6800000FB0616B3586FEA03536FEA1353B35037
:10A6900017E0242256435B090C22A17802FB0363D6
:10A6A000E27842EA01220B495B185A6009E0242251
:10A6B00056435B090C2202FB03630649E2785B18F0
:10A6C0001A72F8BD540B0020C40B0020BC0B0020F4
:10A6D000C80B0020000B00202DE9F3414901CEB248
:10A6E00001AC46F015031746694622468DF8043042
:10A6F0008046FFF75BFF9DF801C09DF8033046F0F0
:10A7000014064046694622466D468DF804608DF871
:10A7100005C08DF806708DF80730FFF747FFBDE8DC
:10A72000FC8100BF2DE9F3414901CEB201AC46F0F6
:10A7300015031746694622468DF804308046FFF718
:10A7400035FF9DF801C09DF8023046F014064046E2
:10A75000694622466D468DF804608DF805C08DF877
:10A7600006308DF80770FFF721FFBDE8FC8100BFC0
:10A7700037B541F001030C466A4601A98DF8003057
:10A780000546FFF713FF9DF806009DF8052000021F
:10A790009DF8073040EA0240184310F4000F18BF3C
:10A7A00040F07F405F2C1AD8C4F3411314F01E040C
:10A7B00002D0022C13D106E0032202FB0535084A21
:10A7C0002D01A8580BE0032202FB053520F07F4144
:10A7D000E8B2FFF7B5FE024B03EB051568683EBD16
:10A7E000C40C002007B541F001036A4601A98DF8A9
:10A7F0000030FFF7DBFE9DF806009DF8073043EAC6
:10A80000002010F4006F1CBF6FEA00506FEA105078
:10A810000EBD00BF13B541F00103144601A96A46FD
:10A820008DF80030FFF7C2FE9DF805109DF8063048
:10A830009DF807202170A27063709DF804001CBD74
:10A8400007B5410141F0160101F0F601002001AA0F
:10A85000FFF7E0FF9DF80530D80913F0200F18BF6F
:10A8600040F002000EBD00BF07B5410141F01601E6
:10A8700001F0F601002001AAFFF7CCFF9DF805309A
:10A88000C3F3801013F0100F18BF40F002000EBD8C
:10A8900037B50C4641EA401101AA0546C9B200206D
:10A8A000FFF7B8FFB4235D436408032305F5807503
:10A8B00003FB04549DF804102046FDF751FA601C78
:10A8C0009DF80510FDF74CFAA01C9DF80610FDF749
:10A8D00047FA3EBD5F292DE9F3410D460646144671
:10A8E00062D8C1F3411811F01E0102D002295BD1D8
:10A8F0001EE0032202FB0088344A4FEA0810831846
:10A900005B688450E01A0028B8BF4042B0F5000FE1
:10A910000ADB9C42CCBF2E4C2E4C2C4A1C1902EB5D
:10A920000812012313733FE002EB081211733BE09E
:10A93000032707FB0087254B3801C1587A00C4EB79
:10A94000010C0132BCF1000FB8BFCCF1000C00EBE0
:10A95000030EBCF5000F24F07F40CEF8044043F80E
:10A9600032001DDBA142CCBF194B1A4B4FEA4818ED
:10A97000E3184FEA234E4FEA232C3046694601AADA
:10A980008DF807308DF804808DF805E08DF806C04D
:10A99000FFF70CFE0D4B03EB071701233B7303E09E
:10A9A00003EBC20300221A714FEA244C23123046F3
:10A9B000694601AA8DF804508DF805C08DF806305F
:10A9C0008DF80740FFF7F2FDBDE8FC81C40C0020C4
:10A9D000FFFF7F00010080FF38B50D466821044667
:10A9E000FFF7C6FE15B140F0010201E020F00102C0
:10A9F00020466821FFF76EFF38BD00BF07B513463C
:10AA00004FEA222C8DF804104FF0000E694601AA7F
:10AA10008DF805E08DF806C08DF80730FFF7C6FD0C
:10AA20000EBD00BF07B50B4611F01E01024601D056
:10AA3000022905D1104619460022FFF74BFF0DE011
:10AA40004FF0000C694601AA8DF804308DF807C05C
:10AA50008DF805C08DF806C0FFF7A8FD0EBD00BF3C
:10AA600010B5C4B22146640100200222E4B2FFF70F
:10AA700059FE002044F00801FFF7D4FF44F00A011A
:10AA80000020FFF7CFFF10BD07B59DF810C08DF86F
:10AA900004108DF80520694601AA8DF806308DF85E
:10AAA00007C0FFF783FD0EBD30B5430185B00446F6
:10AAB00043F00303002003A902AA8DF80830FFF732
:10AAC00075FD9DF80E109DF80D209DF80F300902C0
:10AAD00041EA024119432046FFF732FD174B03EBD1
:10AAE000041108310A7932B3154A0C2000FB042204
:10AAF000107A00BB2201D518D2586B68C3EB020C48
:10AB0000BCF1000FB8BFCCF1000CBCF5000F05DBA9
:10AB10009A42CCBF0B4A0C4A9A1800E008716101B6
:10AB2000C2F30723D4B201F0E0010020C2F30742D0
:10AB30000094FFF7A9FF05B030BD00BFC40C002092
:10AB4000000B0020FFFF7F00010080FF07B5937816
:10AB500092F800E092F801C08DF8041001AA69464D
:10AB60008DF805E08DF806C08DF80730FFF71EFD63
:10AB70000EBD00BF37B5440144F01604E4B20D46E3
:10AB800001AA21460020FFF745FE9DF8053015F08B
:10AB9000010F1ABF6FEA43636FEA536303F07F0349
:10ABA0008DF805309DF8053015F0020F14BF43F005
:10ABB000200323F020038DF805300023184621469A
:10ABC00001AA8DF80630FFF7C1FF3EBD37B544013D
:10ABD00044F01604E4B20D4601AA21460020FFF716
:10ABE00019FE9DF8053015F0010F14BF43F0400326
:10ABF00023F040038DF805309DF8053015F0020F65
:10AC000014BF43F0100323F010038DF80530002328
:10AC10001846214601AA8DF80630FFF797FF3EBD82
:10AC200073B5B42545434B08032205F5807502FB37
:10AC30000355044628460E46FCF7FCFF8DF8040039
:10AC4000681CFCF7F7FF8DF80500A81CFCF7F2FF65
:10AC500046EA44148DF80600E1B2002001AAFFF78D
:10AC600075FF7CBD2DE9F74F4001C7B24C050020B0
:10AC700047F0180101AAFFF7CDFD9DF80560640DAE
:10AC800006F00F053609B5420EDB204604F0C4FB82
:10AC9000AD1B80460120A840894604F0CDFB002270
:10ACA000334B04F02FFC0FE0204604F0B5FB751B7E
:10ACB00080460120A840894604F0BEFB02460B46B0
:10ACC00000202B4904F048FD02460B464046494609
:10ACD00004F042FD04F050FE04F0C0FB22A3D3E9CF
:10ACE000002304F00FFC04F047FE04F0B7FB002241
:10ACF000204B04F007FC4FF0FF36B046002582469B
:10AD00008B460120A84004F097FB02460B465046B4
:10AD1000594604F0F7FB04F007FEA0F180027F2AF9
:10AD200098BF2E46034605F1010588BF43460E2D08
:10AD300001D09846E5E7002547F0120101AA284610
:10AD40008DF805308DF806608DF80450FFF7FEFE93
:10AD5000284647F00C012246FFF750FE2846BDE882
:10AD6000FE8F00BFAFF3008004560E2DB29DEF3F63
:10AD7000000060400000204013B5154B587E10F0D5
:10AD8000010003D000206821212201E06821202257
:10AD90000024FFF79FFD20467E21202223460094B9
:10ADA000FFF772FEE1B200200134FFF739FF1D2CDE
:10ADB000F8D10C210020FFF7DBFC01460020FFF753
:10ADC00051FF0020162143F2FF12FFF717FE1CBDB2
:10ADD00004000020AFF30080084B1868034605E02C
:10ADE0002C2A02D100221A7003E001331A78002ABB
:10ADF000F6D1024A01331360704700BF940400206B
:10AE000010B50E4B02461B78ABB10D4B1C7994B1BB
:10AE10009C68601CE4180D2A2273986002D03F28B9
:10AE200000D851B9064C014604F10C00FDF7EAFCCC
:10AE30000023A36001E0FDF787F910BDD00A0020D0
:10AE40009404002030B50121044687B02020FFF78C
:10AE5000D7FF002C04DA2D200121FFF7D1FF644237
:10AE600000230A2194FBF1F201FB124101AD3031C4
:10AE7000E954591C141E01DD0B46F2E7ED181C467F
:10AE80000121013C15F80109FFF7BAFFB4F1FF3FBA
:10AE9000F6D107B030BD00BF38B50C4D0446A878D8
:10AEA00001214030C0B2FFF7ABFF6878012140308C
:10AEB000C0B2FFF7A5FF2078FFF7C4FF6068FFF777
:10AEC000C1FF0D200121FFF79BFF38BD04000020CA
:10AED00070B5124B06461B78EBB1FDF703F9104C29
:10AEE000054618B100232371012016E0E36C226DA2
:10AEF000934208D21A1992F854200133012032707B
:10AF0000E364207109E004F15400FDF749FCE564B5
:10AF10002065284601E0FDF7E5F870BDD00A002065
:10AF2000940400202DE9F34104460DF10700FFF7DA
:10AF3000CFFF002800F0CB808B4B8C4A93F8941005
:10AF400019BB51789DF80700403188420DD1D3F8E4
:10AF50009810002940F0BB801179012231F00101E5
:10AF600083F8942040F0B380AFE00D2801D01B2877
:10AF700002D100227C4B05E0D3F898207E2A00F213
:10AF8000A6800132C3F89820A1E0117931F00101C7
:10AF900003D19DF80700FFF733FF9DF807301F2B03
:10AFA0000BD9714AD2F898107E297FD8481C89188D
:10AFB00081F89C30C2F8980078E0082B08D16A4BE1
:10AFC000D3F89820002A71D0013AC3F898206DE098
:10AFD0000D2B6BD1644BD3F89830002B66D0634BAC
:10AFE0001A79112A15D1587801214030C0B2FFF7E3
:10AFF00007FF002503E0585DFFF702FF01355A4BBC
:10B000000121D3F898209C339542F4D30D20FFF70B
:10B01000F7FE554A00231568D2F8987019461A466B
:10B0200033E001290FD002D302292DD122E04E4E68
:10B0300006F19C00805C202826D09E1986F81C0111
:10B040000133012120E0484800F19C0C1CF802C0AB
:10B05000BCF1200F0AD1012B04D91818002180F867
:10B060001C110133424D0221ED180DE0181880F833
:10B070001CC108E03C4E06F19C00805C202803D0F7
:10B080009E1986F81C0101330132BA42C9D3364AEF
:10B090000021981880F81C110120C2F89810156042
:10B0A00082F8A001C2F89C3182F894109DF8073014
:10B0B0001B2B0CD12D4A2C4B12790021012A83F82D
:10B0C0009410C3F8981002D10D20FFF799FE264B7B
:10B0D00093F8A001002878D00022164683F8A0211A
:10B0E0001546DFF8A880072707FB05872048394663
:10B0F000013503F023FE30B9BE797B7916F0010FDC
:10B10000237049D007E018F806300736002B5ED0D0
:10B11000FF2DE6D15BE0FFF75FFE23780546042BA9
:10B120000CD1144903F00AFE0346D8B1284612494F
:10B1300003F004FE70B1284610490FE00D2B28D112
:10B140000F4903F0FBFD034660B128460D4903F0AB
:10B15000F5FD08B9012305E00B49284603F0EEFD93
:10B16000B0B90223637017E09404002004000020AB
:10B17000B0050020090301080D03010811030108AF
:10B18000170301081D030108220301080801010833
:10B19000284603F0CDFD607016F0020F04D0FFF7D3
:10B1A0001BFE03F0C5FDA07016F0040F0CD0FFF7D6
:10B1B00013FE03F0BDFD010EC0F30722C0F30743E9
:10B1C000A17122716371E0700120BDE8FC81002350
:10B1D0002370F9E7704700BFFEE700BFFEE700BF3E
:10B1E000FEE700BFFEE700BF704700BF704700BF2B
:10B1F000704700BF704700BF704700BF704700BF77
:10B20000704700BF704700BF704700BF704700BF66
:10B21000704700BF704700BF704700BF704700BF56
:10B22000704700BF704700BF704700BF704700BF46
:10B23000704700BF704700BF704700BF704700BF36
:10B2400008B5024B1B68984708BD00BFF00A0020F4
:10B2500008B5024B1B68984708BD00BFC00B002013
:10B2600008B5024B1B68984708BD00BF500B002073
:10B2700008B5024B1B68984708BD00BF740B00203F
:10B28000704700BF704700BF704700BF704700BFE6
:10B29000704700BF704700BF704700BF704700BFD6
:10B2A000704700BF704700BF704700BF704700BFC6
:10B2B000704700BF704700BF704700BF704700BFB6
:10B2C000704700BF704700BF704700BF704700BFA6
:10B2D000704700BF704700BF704700BF704700BF96
:10B2E000704700BF704700BF704700BF704700BF86
:10B2F000704700BF704700BF704700BF704700BF76
:10B30000704700BF704700BF704700BF704700BF65
:10B31000704700BF436830B523F470230C680A7986
:10B3200023F48073234343EA0223436082688D68D9
:10B33000CC680A4B45EA040C02EA03034A794CEA5A
:10B34000030343EA420383600B7CC26A013B22F49D
:10B350007002DBB242EA0353C36230BDFDF7F1FF76
:10B36000002301220274C360036003714371836090
:10B37000704700BF19B1836843F0010302E083689E
:10B3800023F001038360704719B1836843F480732D
:10B3900002E0836823F4807383607047C9B212B1FE
:10B3A0004368194302E0436823EA010141607047A2
:10B3B000836843F008038360704700BF8068C0F370
:10B3C000C0007047836843F004038360704700BF88
:10B3D0008068C0F38000704719B1836843F4A0030C
:10B3E00002E0836823F4A003836070478068C0F3A1
:10B3F000805070474368013923F4604343EA413386
:10B400004360704719B1436843F4006302E0436846
:10B4100023F4006343607047092930B511D94FF018
:10B42000030C0CFB01FC0725ACF11E0C05FA0CF516
:10B4300003FA0CFCC46824EA050343EA0C03C36066
:10B440000EE04FF0030C0CFB01FC072505FA0CF590
:10B4500003FA0CFC046924EA050343EA0C030361C4
:10B46000062A0DD80523013A5A434FF01F0C0CFA57
:10B4700002FC9140436B23EA0C020A4342631CE046
:10B480000C2A0DD805235A434FF01F0C233A0CFA0F
:10B4900002FC9140036B23EA0C020A4302630CE0B6
:10B4A00005235A434FF01F0C413A0CFA02FC91401D
:10B4B000C36A23EA0C020A43C26230BD19B1836831
:10B4C00043F4801302E0836823F4801383607047A1
:10B4D000C06C80B2704700BF014B1868704700BF56
:10B4E0004C24014019B1436843F4806302E043688F
:10B4F00023F480634360704719B1436843F4805379
:10B5000002E0436823F4805343607047836823F468
:10B51000E04341EA03038360704700BF19B18368C9
:10B5200043F4004302E0836823F4004383607047E0
:10B5300019B1836843F4021302E0836823F4021311
:10B54000836070478068C0F340507047092930B568
:10B5500011D94FF0030C0CFB01FC0725ACF11E0CBC
:10B5600005FA0CF503FA0CFCC46824EA050343EA67
:10B570000C03C3600EE04FF0030C0CFB01FC07252D
:10B5800005FA0CF503FA0CFC046924EA050343EA06
:10B590000C030361836BC3F3015CCCEB0202023248
:10B5A0004FF0050CD2B20CFB02F20CF11A0C0CFAA3
:10B5B00002FC914023EA0C030B43836330BD00BFC0
:10B5C000836B013923F4401343EA015383637047CB
:10B5D0000A5070472830405880B27047436823F4BF
:10B5E000400323F4007341EA03034360704700BF44
:10B5F00041628262704700BF436823F01F0341EA43
:10B6000003034360704700BF20B1054B9A6842F4C2
:10B61000000203E0024B9A6822F400029A6070472D
:10B6200000240140036819420CBF0020012070472C
:10B63000C9430160704700BF4368006810EA1120E9
:10B6400004D0C9B219420CBF00200120704700BFCE
:10B650006FEA11210160704708B5134B98420FD073
:10B6600003F5A053984213D0A3F5C053984219D1C3
:10B670004FF40070012100F0F3FF4FF400700EE072
:10B680004FF48060012100F0EBFF4FF4806006E092
:10B690004FF40040012100F0E3FF4FF4004000218F
:10B6A00000F0DEFF08BD00BF002801400268002353
:10B6B00022F001020260036043608360C3602D4B8F
:10B6C000984233D011D83C3B984229D006D8283B29
:10B6D000984221D0143398424BD11FE0264B984218
:10B6E00020D01433984244D11EE0244B98422CD0F1
:10B6F00008D8A3F5677398421DD003F5627398428A
:10B7000037D11DE01E4B984229D0143398422BD0DC
:10B71000283B98422DD11DE01A4B12E0194B15E041
:10B72000184B18E0174B1BE0164B1EE0154B5A68E0
:10B7300042F470021CE0134B5A6842F0706217E04A
:10B74000114B5A6842F00F0212E00F4B5A6842F058
:10B75000F0020DE00C4B5A6842F4706208E00A4BAC
:10B760005A6842F4704203E0074B5A6842F4702270
:10B770005A6070476C000240440002401C040240C2
:10B780004404024000000240000402408A6870B590
:10B790000C6A0B6944EA02024C691A438B69224322
:10B7A000CC6905684E6A42EA030323438C6A33433B
:10B7B00025F4FE4C23432CF0F00C43EA0C03036009
:10B7C000CB6843600B6883604B68C36070BD00BF8B
:10B7D00000238362036043608360C360036143614D
:10B7E0008361C36103624362704700BF19B103689C
:10B7F00043F0010302E0036823F001030360704794
:10B8000012B10368194302E0036823EA01010160F1
:10B81000704700BF406880B2704700BF10F0805F83
:10B8200014BF044B044B1B6803420CBF00200120D3
:10B83000704700BF000402400000024010F0805F2B
:10B8400014BF024B024B5860704700BF0004024017
:10B850000000024010F0805F14BF044B044B1B68D3
:10B8600003420CBF00200120704700BF00040240CB
:10B870000000024010F0805F14BF024B024B586082
:10B88000704700BF0004024000000240044B002249
:10B890001A605A609A60DA60024A5A61704700BFC3
:10B8A00000040140FFFF0700837930B50168027989
:10B8B0004BB3184BCC431D6890F805C004EA05054E
:10B8C0001D605D682C405C60D45844EA0101D15091
:10B8D00002689868D14301EA00009860D868014086
:10B8E000BCF1100FD96007D1996811439960D968EC
:10B8F00041EA0202DA600BE05CF8031041EA02025E
:10B900004CF8032004E0034BD05820EA0101D15049
:10B9100030BD00BF0004014000230C22837142713E
:10B9200003600371704700BF024B1A6940EA0202CC
:10B930001A61704700040140034B5B6918420CBF59
:10B9400000200120704700BF00040140014B5861F6
:10B95000704700BF00040140054B1A685B69034053
:10B9600001D1184603E010420CBF002001207047AF
:10B9700000040140014B5861704700BF00040140C2
:10B98000044B1A6802F038021A601A6840EA020290
:10B990001A60704700200240044B1A6822F0080227
:10B9A0001A601A6840EA02021A60704700200240DA
:10B9B000044B1A6822F010021A601A6840EA020268
:10B9C0001A60704700200240034B044A5A6002F19B
:10B9D00088325A60704700BF00200240230167454B
:10B9E000024B1A6942F080021A617047002002403F
:10B9F000014BD8698008704700200240014B186A4B
:10BA0000704700BF00200240024BD869C0F34000DD
:10BA1000704700BF00200240024B1868C0F340107E
:10BA2000704700BF0020024019B1054B1A6910434E
:10BA300003E0034B1A6922EA00001861704700BF57
:10BA400000200240012804D1054BD86900F0010014
:10BA500005E0034BDB6818420CBF00200120704753
:10BA600000200240014BD860704700BF0020024018
:10BA7000094BDA6812F0010F01D001200BE0DA68FF
:10BA800012F0040F01D0022005E0DB6813F0100F64
:10BA900014BF0320042070470020024013B5044661
:10BAA0000AE000230193FF3301E0019B013B019376
:10BAB000019B002BF9D1013CFFF7DAFF012802D1ED
:10BAC000002CEED100E004B905201CBDF8B5124CE5
:10BAD000124B0546A36003F188330F20A3600E4686
:10BAE0001746FFF7DBFF042814D1236945F0F8055A
:10BAF00043F0100323612E43094B37430B305F8023
:10BB0000FFF7CCFF012805D0226941F6EF7302EA66
:10BB100003032361F8BD00BF0020024023016745F5
:10BB200000F8FF1F38B5054640F6FF70FFF7B6FF77
:10BB300004283CD11E4C1F4B40F6FF70A36003F15C
:10BB40008833A360236943F020032361236943F012
:10BB500040032361FFF7A2FF042820D1226941F6A8
:10BB6000DF7302EA03032361236943F010032361B7
:10BB70001DB1114B4FF0000202E00F4B4FF0A50238
:10BB80001A8040F6FF70FFF789FF01280FD0084A9E
:10BB900041F6EF73116901EA0303136107E001281D
:10BBA00005D0226941F6DF7302EA0303236138BD41
:10BBB000002002402301674500F8FF1F10B504462E
:10BBC0000F20FFF76BFF04283DD11F4A1F4BE443B2
:10BBD000936003F1883393601169E3B241F010017F
:10BBE000FF2B116106D01A4A0B301381FFF756FF65
:10BBF00004281FD1C4F30723FF2B06D0144A0F20BB
:10BC00005381FFF74BFF042814D1C4F30743FF2BE4
:10BC100006D00F4A0F209381FFF740FF042809D177
:10BC2000240EFF2C01D1042006E0094B0F20DC81FB
:10BC3000FFF734FF012806D0034A41F6EF7311697C
:10BC400001EA0303136110BD002002402301674590
:10BC500000F8FF1F70B504460F200E46FFF71EFFC9
:10BC6000042815D10B4D0C4B0B30AB6003F188331E
:10BC7000AB602B6943F010032B612680FFF70EFFAA
:10BC8000012805D02A6941F6EF7302EA03032B610C
:10BC900070BD00BF002002402301674570B5044617
:10BCA0000F200E46FFF7FAFE042810D1084D0B3086
:10BCB0002B6943F001032B612680FFF7EFFE01287B
:10BCC00005D02A6941F6FE7302EA03032B6170BDB9
:10BCD0000020024070B504460F200E46FFF7DEFE3E
:10BCE000042818D10C4DB3B22A690B3042F001027E
:10BCF0002A612380FFF7D2FE042804D1360C668027
:10BD00000B30FFF7CBFE012805D02A6941F6FE7300
:10BD100002EA03032B6170BD0020024010B540F61B
:10BD2000FF70FFF7BBFE04282CD1174C174B40F6D1
:10BD3000FF70A36003F18833A360236943F02003FD
:10BD40002361236943F040032361FFF7A7FE042822
:10BD500010D1226941F6DF7302EA030323612369EC
:10BD60004FF0A50243F010032361094B0B301A80FA
:10BD7000FFF794FE012805D0226941F6EF7302EA2D
:10BD80000303236110BD00BF00200240230167456B
:10BD900000F8FF1F10B540F6FF70FFF77FFE042884
:10BDA00014D10B4C40F6FF70236943F00403236168
:10BDB000236943F040032361FFF770FE012805D09B
:10BDC000226941F6FB7302EA0303236110BD00BF41
:10BDD0000020024038B5054640F6FF70FFF75EFED2
:10BDE000042815D10B4C40F6FF70236943F0020381
:10BDF00023616561236943F040032361FFF74EFE31
:10BE0000012805D0226941F6FD7302EA030323618C
:10BE100038BD00BF00200240CB78F0B513F0100F02
:10BE200018BF8A78098803F00F0C18BF4CEA020C7F
:10BE300011F0FF0F1AD0046800220126964006EA8E
:10BE40000105B5420ED196000F27B7400CFA06F651
:10BE500024EA07043443282B01D1456102E0482B32
:10BE600008BF05610132082AE7D10460FF291CD907
:10BE70004468002202F108050126AE4006EA0105E9
:10BE8000B5420ED196000F27B7400CFA06F624EA09
:10BE900007043443282B01D1456102E0482B08BF39
:10BEA00005610132082AE5D14460F0BD0423C37066
:10BEB000022383704FF0FF33038070478368194279
:10BEC0000CBF002001207047806880B2704700BF1F
:10BED000C36819420CBF002001207047C06880B2BF
:10BEE000704700BF01617047416170470AB101614D
:10BEF00000E04161704700BFC160704741F480338A
:10BF0000836181618361836983697047064A10B5E3
:10BF100014684FF6807341EA001104EA030341EA12
:10BF20000303136010BD00BF00000140014B186007
:10BF3000704700BF1C0020420304154A00F4401C57
:10BF40001B0CBCF5401F30B5546806D1556824F071
:10BF5000706425F07065556011E010F4801F06D004
:10BF6000C0F303424FF0030C0CFA02F203E0420D5F
:10BF7000120113FA02F224EA020444F0706419B1C7
:10BF8000400D000183401C43014B5C6030BD00BF8D
:10BF90000000014001F003039B000F229A4010FAB9
:10BFA00003F310B58908074C023154F8210020EA48
:10BFB000020244F8212054F82120134344F8213090
:10BFC00010BD00BF000001400120014608B500F08F
:10BFD00047FB0120002100F043FB08BD08B5264BBC
:10BFE00098422BD00CD8A3F5006398421AD003F5E1
:10BFF000806398421CD0A3F5006398423AD10BE0CD
:10C000001E4B984226D003F58063984228D0A3F5B2
:10C01000006398422ED117E00420012100F020FB9C
:10C02000042024E00820012100F01AFB08201EE073
:10C030001020012100F014FB102018E02020012125
:10C0400000F00EFB202012E04020012100F008FB50
:10C0500040200CE08020012100F002FB802006E05F
:10C060004FF48070012100F0FBFA4FF48070002142
:10C0700000F0F6FA08BD00BF00140140001C0140AA
:10C080000B4B4FF0FF316FF07042C3F88010C3F8D4
:10C090008420C3F88011C3F88421002303F1C00178
:10C0A000034A013300200F2B42F82100F6D17047DC
:10C0B00000E100E0094B4FF0206058600848002282
:10C0C0004FF0FF319A60D8601A615A619A61DA6163
:10C0D0001A625A629962D9621963704700ED00E0F2
:10C0E0000000FA0540F0BE60024B40F42020D8600A
:10C0F000704700BF00ED00E030B5C27803787AB336
:10C100001C4A4178D2684FF00F0CD243C2F302228E
:10C110002CFA02FCC2F104029140807803F0030281
:10C120000CEA000C4CEA010CD2004FEA0C1CFF2078
:10C1300090400CFA02FC012403F01F02944099087D
:10C140000D4AC03152F821500CEA000C25EA0000DB
:10C150004CEA00005B0942F8210042F8234008E065
:10C1600003F01F02012191405B09034A203342F88A
:10C17000231030BD00ED00E000E100E00023C370BB
:10C180000370437083707047024B5868C0F30930E6
:10C19000704700BF00ED00E0012200F01F0312FA1B
:10C1A00003F34009044A403052F8200018409842F6
:10C1B00014BF00200120704700E100E0014B18602F
:10C1C000704700BF00EF00E000F01F0301229A401B
:10C1D0004009024B603043F82020704700E100E046
:10C1E000024B58688005800D704700BF00ED00E0ED
:10C1F000012200F01F0312FA03F34009044A8030C1
:10C2000052F820001840984214BF002001207047C7
:10C2100000E100E0014B1868704700BF00ED00E04E
:10C2200021F0604121F07F01014B0143996070478B
:10C2300000ED00E0014A024BDA6070470400FA05A5
:10C2400000ED00E0014A024BDA6070470100FA0598
:10C2500000ED00E019B1054B1A69104303E0034BF0
:10C260001A6922EA00001861704700BF00ED00E083
:10C2700000F01F00012313FA00F019B1044B5A6AB1
:10C28000104303E0024B5A6A22EA000058627047EA
:10C2900000ED00E0144B70B5DC684FF0FF0CE44398
:10C2A000C4F302242CFA04F5C4F1040411FA04F4D2
:10C2B000C0F30126F6000CFA06FC02EA050545EA81
:10C2C0000404240114FA06F6C0F38110063053F872
:10C2D000202022EA0C0243F8202053F820201643A5
:10C2E00043F8206070BD00BF00ED00E0C0F3832084
:10C2F00001238340044A506A03EA0000984214BFB5
:10C3000000200120704700BF00ED00E000F01F009A
:10C3100001228240024B59680A435A60704700BFAD
:10C3200000ED00E000F01F020123013A13FA02F2CF
:10C33000024B59680A435A60704700BF00ED00E0A5
:10C34000C0F3833001238340044A506A03EA0000AB
:10C35000984214BF00200120704700BF00ED00E0AC
:10C36000C0F3814313B90A4BD86A10E0012B0CD1FA
:10C37000074AC0F30153906ADA00D040022B14BF81
:10C3800000F00F0000F0FF0001E0014B186B704758
:10C3900000ED00E010F4800F0BBF024B014B586B17
:10C3A000986B704700ED00E008B5F7F7E1FE08BDB7
:10C3B00008B50001F7F7D9FE08BD00BF08B5F7F7CB
:10C3C000D2FE08BD08B5F7F7CCFE08BD08B5F7F7F3
:10C3D000C6FE08BD08B5F7F7C0FE08BD0D4B0E4AF6
:10C3E000196841F001011960596801EA02025A60B6
:10C3F0001A6822F0847222F480321A601A6822F4D9
:10C4000080221A605A6822F4FE025A6000229A6062
:10C41000704700BF001002400000FFF80C4BB0F561
:10C42000803F1A6822F480321A601A6822F480224F
:10C430001A6003D0B0F5802F08D103E01A6842F4E7
:10C44000803202E01A6842F4A0221A60704700BFEE
:10C4500000100240034B1A6822F0F80242EAC002C0
:10C460001A60704700100240014B1860704700BF0F
:10C4700000004242044B5A6822F47C1240EA020255
:10C480000A435A60704700BF00100240014B186019
:10C49000704700BF60004242034B5A6822F003021B
:10C4A00040EA02025A60704700100240024B58688E
:10C4B00000F00C00704700BF00100240034B5A68A8
:10C4C00022F0F00240EA02025A6070470010024077
:10C4D000034B5A6822F4E06240EA02025A60704755
:10C4E00000100240034B5A6822F4605242EAC00234
:10C4F0005A6070470010024019B1054B1A7810437A
:10C5000003E0034B1A7822EA00001870704700BF5E
:10C5100009100240014B1860704700BFD80042422A
:10C52000034B5A6822F4404240EA02025A607047C4
:10C5300000100240064B002201281A701A7002D027
:10C54000042804D101E0187001E005221A70704738
:10C5500020100240014B1860704700BF8004424227
:10C56000024B1A6A40EA02021A6270470010024047
:10C57000014B1860704700BF3C0442421F4B10B58E
:10C580005A6802F00C02042A13D0082A11D15A6802
:10C590005968C2F38342023211F4803F03D05B68D2
:10C5A00013F4003F01D0164B00E0164B5A430260D3
:10C5B00001E0144B0360114A134B51680468C1F346
:10C5C0000311595C34FA01F141605468C4F3022C40
:10C5D00013F80C4031FA04F484605468C4F3C22C9C
:10C5E00013F80CC021FA0CF1C1605268C2F3813219
:10C5F0009B181B7CB1FBF3F1016110BD00100240E0
:10C6000000093D0000127A00E801010819B1054B4C
:10C610005A69104303E0034B5A6922EA000058614B
:10C62000704700BF0010024019B1054B9A691043D2
:10C6300003E0034B9A6922EA00009861704700BF4B
:10C640000010024019B1054BDA69104303E0034BB7
:10C65000DA6922EA0000D861704700BF001002408A
:10C6600019B1054BDA68104303E0034BDA6822EA9C
:10C670000000D860704700BF0010024019B1054BA0
:10C680001A69104303E0034B1A6922EA000018619B
:10C69000704700BF00100240014B1860704700BF98
:10C6A00040044242014B1860704700BF4C004242B8
:10C6B000014B1870704700BF071002404309012B5F
:10C6C00002D1084B1B6805E0022B0BBF054B054B45
:10C6D0001B6A5B6A00F01F0033FA00F000F00100F3
:10C6E000704700BF0010024008B53120FFF7E6FF99
:10C6F000094B18705A6801325A601A7822B95A6880
:10C7000040F2FF139A42F0D13120FFF7D7FF0038F3
:10C7100018BF012008BD00BF38060020024B5A6A2E
:10C7200042F080725A62704700100240034B9B68CF
:10C7300018420CBF00200120704700BF00100240CB
:10C74000014B1870704700BF0A1002400B884A88DE
:10C75000B1F804C01A43CB8842EA0C02B1F808C011
:10C760001A434B8930B542EA0C028D89B0F800C0FB
:10C77000CC891A432A4322430CF4415313439BB2FE
:10C780000380838B23F400631B041B0C83830B8ABD
:10C79000038230BD00234FF00702C3810282038071
:10C7A00043808380C380038143818381704700BFBE
:10C7B00000234381038043808380C3804FF00203C2
:10C7C0000381704721B103889BB243F0400304E02A
:10C7D000038823F040031B041B0C0380704700BF39
:10C7E00021B1838B9BB243F4806304E0838B23F4F9
:10C7F00080631B041B0C8383704700BF090901235E
:10C8000013FA01F189B21AB183889BB2194303E08C
:10C8100083889BB223EA0101818070471AB1838823
:10C820009BB2194303E083889BB223EA0101818014
:10C83000704700BF81817047808980B2704700BF18
:10C840004FF6FF63994205D003889BB243F480738F
:10C85000038002E0038819400180704721B183887A
:10C860009BB243F0040304E0838823F004031B0419
:10C870001B0C8380704700BF038823F400631B04F4
:10C880001B0C038003889BB241EA030303807047BB
:10C8900003889BB243F480530380704721B103881F
:10C8A0009BB243F4005304E0038823F400531B04B9
:10C8B0001B0C0380704700BF012914BF008B808AC6
:10C8C00080B27047008A80B2704700BFB1F5804FD8
:10C8D00004D103889BB243F4804304E0038823F42B
:10C8E00080431B041B0C0380704700BF038919425F
:10C8F0000CBF002001207047202906D1038903883E
:10C900009BB243F04003038008E0402901D008298E
:10C9100001D1038902E0C94389B20181704700BF98
:10C92000012301F00F0213FA02F2B0F804C00089EB
:10C930001FFA8CFC80B2104006D009098B401CEA1B
:10C94000030F0CBF00200120704700BF552906D1FE
:10C95000038903889BB243F0400303800DE056290E
:10C9600001D0532901D1038907E001F00F01012310
:10C9700013FA01F1C94389B201817047838BF0B585
:10C9800023F47A6323F01F031B041B0C83834FF0F3
:10C99000020303840B89868B022B87B004460D4665
:10C9A000B6B201D1002225E001A88F88FFF7E6FD8D
:10C9B000EB88002F0CBF01270227B3F5007F2989E0
:10C9C000019A06D1A3F5FB7353430902B3FBF1F3BC
:10C9D00005E00A2349015A434F43B2FBF7F30533FD
:10C9E0000A229BB2B3FBF2F303F001021202C3F37B
:10C9F0004F0392B2991E89B2FE2928BF002228BF98
:10CA00000223E98842EA03030B439BB223842B8869
:10CA10006A8846EA0303A98843F4006313436A89DA
:10CA20000B4313439BB2A38307B0F0BD08B5154B6E
:10CA300098421BD003F57443984204D0A3F5784381
:10CA400098421DD10AE001214FF48050FFF708FE03
:10CA50004FF480500021FFF703FE11E04FF48040B7
:10CA60000121FFF70BFE4FF4804006E04FF4004039
:10CA70000121FFF703FE4FF400400021FFF7FEFD08
:10CA800008BD00BF003C0040042804D1054B1A68D3
:10CA900042F0040203E0034B1A6822F004021A6019
:10CAA000704700BF10E000E0014B5860704700BFC6
:10CAB00010E000E0012804D1084B1A6842F001029E
:10CAC00006E010F1020F05D1044B1A6822F00102B2
:10CAD0001A6002E0014B00229A60704710E000E00B
:10CAE00020B1054B1A6842F0020203E0024B1A68BB
:10CAF00022F002021A60704710E000E0014B9868D3
:10CB0000704700BF10E000E0C308022B0BBF044BCE
:10CB1000034B1B68DB6833FA00F000F0010070473C
:10CB200010E000E0038803F08F0303800388B1F86E
:10CB300006C04A889BB243EA0C0313439BB20380AE
:10CB40008B8883850B880385064B984203D003F5B9
:10CB50000063984201D10B7A03864FF00103838270
:10CB6000704700BF002C0140038C2DE9F04123F0F9
:10CB700001031B041B0C0384038C0A894C8823F0DB
:10CB800002031C4E14431B048288B1F806C0058BB7
:10CB90001B0CA4B2B04244EA030392B20C88ADB2BB
:10CBA000A0F834C003D006F50066B04218D18E89D3
:10CBB0004F89B1F80E804FF6F77C03EA0C0C4CEA73
:10CBC000070748EA06064FF6FB73898847F6FF4CCD
:10CBD00002EA0C0C07EA0303B2B20B4342EA0C026E
:10CBE0004FF68F7105EA010121438280018303849E
:10CBF000BDE8F081002C0140038C2DE9F04123F0C9
:10CC000010031B041B0C0384028CB1F808C022F033
:10CC1000200212048488120C4B8842EA0C1242EA69
:10CC20000313A2B21B4C068BB1F806C0A0420D88BC
:10CC3000B6B29BB2A0F838C003D004F50064A0429D
:10CC40001BD1B1F80A804FF67F748F8903EA040480
:10CC500047F2FF3C02EA0C0C44EA0814CA894FF67A
:10CC6000BF73898804EA03034CEA870C43EA011383
:10CC70004CEA82023C469BB292B248F6FF7106EA49
:10CC8000010141EA052189B2828001830384BDE864
:10CC9000F08100BF002C0140038C2DE9F04123F40A
:10CCA00080731B041B0C0384028CB1F808C022F4AF
:10CCB000007212048488120C4B8842EA0C2242EA69
:10CCC0000323A2B21A4C868BB1F806C0A0420D888D
:10CCD000B6B29BB2A0F83CC003D004F50064A042F9
:10CCE0001BD1B1F80A804FF2FF748F8903EA040464
:10CCF00044F6FF7C02EA0C0C44EA0824CA894FF689
:10CD0000FF33898804EA03034CEA071C43EA012342
:10CD10004CEA02123C469BB292B24FF68F7106EA81
:10CD200001012943828081830384BDE8F08100BF33
:10CD3000002C0140038CF0B523F480531B041B0C22
:10CD40000384B1F806C0078C0C8882880D89868B15
:10CD50004B88A0F840C0DFF848C0BFB2604592B22F
:10CD6000B6B203D00CF5006C604505D192048989F8
:10CD7000920C42EA811292B24DF6FF7C07EA0C0C4B
:10CD800048F6FF7106EA01014CEA053C41EA04213C
:10CD90004CEA033389B29BB2828081830384F0BD65
:10CDA000002C0140B1F802C00B888A884CEA0303CA
:10CDB000B1F806C013430A8943EA0C03B1F80AC06C
:10CDC00013438A8943EA0C0313439BB2A0F844300F
:10CDD000704700BF00234FF0FF3203724380828010
:10CDE0000380C380704700BF0023C381038043805A
:10CDF0008380C380038143818381704700234FF088
:10CE000001020381038043808280C380704700BF9A
:10CE100000238381038043808380C3800381438117
:10CE2000704700BF21B103889BB243F0010304E0C7
:10CE3000038823F001039B059B0D0380704700BF0F
:10CE400039B1B0F844306FEA43436FEA53439BB2C1
:10CE500003E0B0F844305B045B0CA0F8443070474A
:10CE60001AB183899BB2194303E083899BB223EAF9
:10CE700001018181704700BF818270470A43A0F899
:10CE8000482070471AB183899BB2194303E0838914
:10CE90009BB223EA01018181704700BF038923F01F
:10CEA00007031B041B0C0381704700BFB0F808C0C8
:10CEB0005FFA8CFC41EA0C0C42EA0C0C4CEA032CA5
:10CEC0001FFA8CFCA0F808C0704700BF10B50446DC
:10CED000FFF7ECFF23899BB243F48043238110BD0D
:10CEE00010B50446FFF7E2FF238923F077031B0404
:10CEF0001B0C43F07703238110BD00BF01858282A4
:10CF0000704700BF038823F070039B059B0D41EA27
:10CF100003030380704700BF038923F070031B04E1
:10CF20001B0C41EA03030381704700BF10B50446A0
:10CF3000FFF7F2FF23899BB243F00703238110BD63
:10CF400030B50489B0F818C0058C2CF4407CADB223
:10CF50002CF0030C24F007044FEA0C4C25F02205BA
:10CF600042EA050524044FEA1C4C45EA0315240C4B
:10CF70004CF4807C21434CF0010CADB20181A0F84F
:10CF800018C0058430BD00BF038B23F070031B0461
:10CF90001B0C41EA03030383704700BF038B23F498
:10CFA000E0431B041B0C43EA01239BB2038370473D
:10CFB000838B23F070031B041B0C41EA0303838360
:10CFC000704700BF838B23F4E0431B041B0C43EA30
:10CFD00001239BB28383704721B103889BB243F046
:10CFE000800304E0038823F080039B059B0D0380EE
:10CFF000704700BF21B183889BB243F0040304E073
:10D00000838823F004031B041B0C8380704700BF3C
:10D0100021B183889BB243F0080304E0838823F0A6
:10D0200008031B041B0C8380704700BF21B1838859
:10D030009BB243F0010304E0838823F001031B0447
:10D040001B0C8380704700BF038B23F008031B0475
:10D050001B0C41EA03030383704700BF038B23F4D7
:10D0600000631B041B0C43EA01239BB2038370473C
:10D07000838B23F008031B041B0C41EA0303838307
:10D08000704700BF838B23F400631B041B0C43EA2F
:10D0900001239BB283837047038B23F004031B049B
:10D0A0001B0C41EA03030383704700BF038B23F487
:10D0B00080631B041B0C43EA01239BB2038370476C
:10D0C000838B23F004031B041B0C41EA03038383BB
:10D0D000704700BF838B23F480631B041B0C43EA5F
:10D0E00001239BB283837047038B23F080031B04CF
:10D0F0001B0C41EA03030383704700BF038B5B04EF
:10D100005B0C43EA01239BB203837047838B23F0BC
:10D1100080031B041B0C41EA03038383704700BF99
:10D12000838B5B045B0C43EA01239BB283837047D0
:10D13000038C23F002031B041B0C41EA030303844A
:10D14000704700BF038C23F008031B041B0C41EA4B
:10D1500003030384704700BF038C23F020031B04E8
:10D160001B0C43EA01139BB203847047038C23F02A
:10D1700080031B041B0C43EA01139BB2038470471A
:10D18000038C23F400731B041B0C43EA01239BB2A2
:10D1900003847047038C23F400631B041B0C43EAD5
:10D1A00001239BB203847047038C23F400531B04B8
:10D1B0001B0C43EA01339BB20384704701238B406D
:10D1C0008A40018C89B221EA03030384018C0A435B
:10D1D00092B20284704700BF04238B408A40018CC6
:10D1E00089B221EA03030384018C0A4392B20284C8
:10D1F000704700BF01238B40B0F820C010B51FFA64
:10D200008CFC2CEA0303038409B1082909D11830E6
:10D21000490844584FF68F7304EA030343504358B8
:10D220000CE004391830C1F34E01445848F6FF733E
:10D2300004EA030343501202435892B243EA020243
:10D24000425010BD21B103889BB243F0020304E0B9
:10D25000038823F002039B059B0D0380704700BFEA
:10D2600021B103889BB243F0040304E0038823F058
:10D2700004039B059B0D0380704700BF21B1838889
:10D280009BB243F0800304E0838823F080031B04F7
:10D290001B0C8380704700BF038823F008039B05A5
:10D2A0009B0D038003889BB241EA03030380704710
:10D2B000838823F070031B041B0C838083889BB23C
:10D2C00041EA030383807047038923F007031B04AB
:10D2D0001B0C038103899BB241EA0303038170475E
:10D2E000038923F080031B041B0C038103899BB279
:10D2F00041EA030303817047818470478185704749
:10D30000818670470187704781877047A0F8401079
:10D31000704700BF038B23F00C031B041B0C03831B
:10D32000038B9BB241EA030303837047038B23F40F
:10D3300040631B041B0C0383038B9BB243EA012352
:10D340009BB20383704700BF838B23F00C031B0445
:10D350001B0C8383838B9BB241EA03038383704757
:10D36000838B23F440631B041B0C8383838B9BB24E
:10D3700043EA01239BB28383704700BF0388DBB27B
:10D38000038003889BB241EA03030380704700BF18
:10D39000808E80B2704700BF008F80B2704700BFA0
:10D3A000808F80B2704700BFB0F8400080B27047F5
:10D3B000808C80B2704700BF008D80B2704700BF84
:10D3C000038A19420CBF002001207047C94389B26B
:10D3D00001827047038A828911EA030092B203D066
:10D3E00011420CBF00200120704700BFC94389B221
:10D3F00001827047B0F820C010B52CF0010C4FEA44
:10D400000C4C4FEA1C4CA0F820C0048BB0F820C094
:10D41000A4B21FFA8CFC24F0F30442EA04042CF0BA
:10D42000020C44EA03144CF0010C4CEA010CA4B2C7
:10D430000483A0F820C010BDB0F820C010B52CF0B7
:10D44000100C4FEA0C4C4FEA1C4CA0F820C0B0F86E
:10D4500018C0048C2CF4407CA4B24FEA0C5C4FEA58
:10D460001C5C24F020044CEA022C44F010044CEA2A
:10D47000033C44EA01141FFA8CFCA4B2A0F818C0C3
:10D48000048410BD38B50D46602D1146044603D105
:10D490000122FFF7D1FF02E00122FFF7ABFF29468F
:10D4A0002046FFF739FD23899BB243F00703238110
:10D4B00038BD00BFF8B50C46A2884988B4F800C052
:10D4C000054600290CBF02270027012A0CBF0226AF
:10D4D00001262389BCF1000F10D1FFF78BFF2846EE
:10D4E000E188FFF717FF2846394632462389FFF7C0
:10D4F000A3FF2846E188FFF719FF0FE0FFF79CFF25
:10D500002846E188FFF712FF28463946324623892C
:10D51000FFF770FF2846E188FFF7FCFEF8BD00BF6B
:10D5200038B50B880C4605464BB94988A288238933
:10D53000FFF760FF2846E188FFF7ECFE53E0042B7D
:10D5400009D14988A2882389FFF776FF2846E18818
:10D55000FFF7ECFE47E0082BB1F802C0B1F804E099
:10D56000098920D1028C22F480721204120C0284E8
:10D57000838B028C9BB292B223F0F30322F40072ED
:10D5800043EA011142EA0C2C89B21FFA8CFC41EAF1
:10D590000E0E4CF4807CA0F81CE0A0F820C0E188BE
:10D5A000FFF7D2FE1FE0028C22F480521204120C0C
:10D5B0000284838B028C23F4407392B21B051B0DF3
:10D5C00022F4005243EA0E2342EA0C3C43EA0133C0
:10D5D0001FFA8CFC9BB24CF4805C8383A0F820C0C3
:10D5E000E188FFF7BDFE38BD08B52D4B984237D016
:10D5F0000BD8A3F50063984226D003F580639842C8
:10D6000028D0B0F1804F4AD118E0264B984233D051
:10D6100004D8A3F58063984241D127E0224B984279
:10D6200004D003F50063984239D12EE04FF4006036
:10D630000121FFF715F84FF400602DE001200146AD
:10D64000FFF71CF801201CE002200121FFF716F86B
:10D65000022016E004200121FFF710F8042010E05A
:10D6600008200121FFF70AF808200AE01020012114
:10D67000FFF704F8102004E020200121FEF7FEFF50
:10D6800020200021FEF7FAFF09E04FF400500121AD
:10D69000FEF7E6FF4FF400500021FEF7E1FF08BD62
:10D6A000000C004000140040002C01400023838146
:10D6B0004FF416528380C38003814FF00C03026045
:10D6C000438170470A8810B54C88B1F804C0038ABA
:10D6D000C98844EA020242EA0C0223F470630A4356
:10D6E0001B041B0C92B242EA0303038210BD00BF6D
:10D6F0000023C380038043808380704721B18389E6
:10D700009BB243F4005304E0838923F400531B04C9
:10D710001B0C8381704700BF01F01F034FF0010C09
:10D72000C1F3421161450CFA03F301D10C3004E05E
:10D73000022901D1103000E014301AB1026842EA27
:10D74000030302E0026822EA03030360704700BF9C
:10D750001AB1838A9BB2194303E0838A9BB223EAFE
:10D7600001018182704700BF038A23F00F031B046D
:10D770001B0C0382038A9BB241EA030303827047B6
:10D78000838923F400631B041B0C838183899BB270
:10D7900041EA03038381704721B183899BB243F03F
:10D7A000020304E0838923F002031B041B0C838122
:10D7B000704700BF038A23F020031B041B0C038265
:10D7C000038A9BB241EA03030382704721B1038AB3
:10D7D0009BB243F4804304E0038A23F480431B0498
:10D7E0001B0C0382704700BFC905C90D81807047BB
:10D7F0008088C005C00D704783899BB243F0010348
:10D8000083817047038BDBB20383038B9BB243EAB4
:10D8100001230383704700BF038B03F47F4303831B
:10D82000038B9BB241EA03030383704721B1838AD0
:10D830009BB243F0200304E0838A23F020031B04FF
:10D840001B0C8382704700BF21B1838A9BB243F0D7
:10D85000100304E0838A23F010031B041B0C838253
:10D86000704700BF21B1838A9BB243F0080304E0F4
:10D87000838A23F008031B041B0C8382704700BFBC
:10D88000838A23F004031B041B0C8382838A9BB2CC
:10D8900041EA03038382704721B1838A9BB243F03C
:10D8A000020304E0838A23F002031B041B0C83821F
:10D8B000704700BF038819420CBF00200120704749
:10D8C000C94389B2018070474FF0010CC1F3421285
:10D8D00001F01F0362450CFA03F301D1828903E0D2
:10D8E000022A0CBF028A828A92B21340028892B244
:10D8F0000BB9184607E0090A012313FA01F1114296
:10D900000CBF002001207047090A01238B40DB4334
:10D910009BB20380704700BF038ACA8823F4405338
:10D920001B041B0C1343038283898A8830B5044689
:10D9300008890D4623F4B053498940EA020223F0D6
:10D940000C030A431B041B0C92B242EA0303A3819B
:10D95000A38AAA8923F440731B041B0C134387B0CA
:10D96000A38201A8FEF70AFE0E4B2A689C420CBF58
:10D97000049B039B1921594392006423B1FBF2F1EC
:10D98000B1FBF3F21201100903FB1011090132314E
:10D99000B1FBF3F303F00F0343EA020292B22281D8
:10D9A00007B030BD0038014008B5214B98422BD05C
:10D9B00008D8A3F50063984216D003F58063984217
:10D9C00034D119E01B4B984226D003F568439842A6
:10D9D0002CD101214FF48040FEF742FE4FF48040ED
:10D9E0000021FEF73DFE21E04FF400300121FEF75B
:10D9F00045FE4FF4003016E04FF480200121FEF781
:10DA00003DFE4FF480200EE04FF400200121FEF790
:10DA100035FE4FF4002006E04FF480100121FEF7A0
:10DA20002DFE4FF480100021FEF728FE08BD00BF38
:10DA3000004C004000500040684620F007018D4631
:10DA400001B5002303E00B495958995004330A4AA1
:10DA50000A4998188842F6D3094B02E0002243F89D
:10DA6000042B084A9342F9D3F6F78AFBBDE801403C
:10DA7000854670473003010800000020280200207E
:10DA800028020020DC0C002010B5074C20B92268C9
:10DA90004FF00103138205E0044B1B681B68984795
:10DAA00020680A3010BD00BF740C0020300C00202C
:10DAB00010B50A4B0A4A1B685178DA7891420AD3AA
:10DAC000997841B99C8834B99A72064B1B685B6897
:10DAD0009847204600E0022010BD00BF740C0020D3
:10DAE00000010020300C002010B5074C20B922683E
:10DAF0004FF00103138205E0044B1B689B689847B5
:10DB000020680C3010BD00BF740C0020300C0020C9
:10DB100038B50E4C0E4B22681B68D1789B69507942
:10DB2000984723689A7A7AB170B91A7962B99D7860
:10DB300055B9084B1B68DB68984723682846597914
:10DB4000DA78D9721A7300E0022038BD740C002014
:10DB50000C0C0020300C002008B50246244B20B9E4
:10DB60001B684FF00201198240E0224A4FF0000189
:10DB70001B681180197811F07F0113D15B7A13F0C3
:10DB8000200F03D0117841F00201117013F0400F03
:10DB9000184B15BF1A781A7822F0010242F00102E0
:10DBA0001A701EE0012921D0022901D000221DE0B7
:10DBB000597911F0800F01F00F0306D00E4951F88A
:10DBC000233003F03003102B06E00B4951F82330CB
:10DBD00003F44053B3F5805F03D1137843F001039E
:10DBE0001370064B1B681B699847024A104608BD14
:10DBF000740C0020D40C0020005C0040300C00208D
:10DC000010B51E4B19684A7912F0800F22F080037C
:10DC100005D01B4850F8230000F0300004E01848FD
:10DC200050F8230000F44050164C94F800C06345AF
:10DC300022D24C8804BBF8B1897AE9B112F0800F86
:10DC400009D00F4948F6BF7251F8230000EA0202DA
:10DC500082F0100208E00A494BF68F7251F8230057
:10DC600000EA020282F4805241F82320064B1B682E
:10DC70009B699847002000E0022010BD740C002032
:10DC8000005C004000010020300C002008B5064B6D
:10DC90001B685A7A42F020025A72044B1B68DB69F7
:10DCA0009847002008BD00BF740C0020300C0020F5
:10DCB000054B1A68538A18B98988CB1A138201E078
:10DCC00008681818704700BF740C002030B50E4B60
:10DCD0001C78002310E05FFA83FC4FEA8C0202F10B
:10DCE000804202F5B842156848F68F7105EA0101D5
:10DCF00041EA0C0111600133A342ECD3034B40F025
:10DD00008000186030BD00BF000100204C5C004066
:10DD1000704700BF08B50C4B002093F82C1000F0A2
:10DD20004FFE0A4B1B68187A082807D1084B4FF49E
:10DD300080521A80074B4FF010021A80092814BF36
:10DD40000020012008BD00BF7C000020740C0020D2
:10DD5000D60C0020D80C002070B52D4B1C68237AFF
:10DD6000032B01D0052B46D1A369228AABB1A2B106
:10DD7000A58A954228BF154628469847228A638A75
:10DD8000521BEB18064622826382002000F0E8FD59
:10DD90002A460146304600F0FBFB238A5BB11D4B4F
:10DDA0004FF4405200201A80014600F0E7FD1A4B64
:10DDB0004FF030021A80A28A238A9A4203D8144B69
:10DDC00003221B6803E0124A1BB1136805221A7272
:10DDD0000DE0126806211172104A1168104A89B2CA
:10DDE0008A18520013600C4B4FF030021A80084B17
:10DDF0001B681B7A06E0072B03D10A4B1B68DB6804
:10DE000098470823024A12681372FFF783FF70BD18
:10DE1000740C0020D60C0020D80C0020505C004070
:10DE2000023000200C0C0020F8B5244B1C68238A1B
:10DE3000267ABBB9042E15D1214822490278012A3D
:10DE40000BD1214C214A24680370A0B282185200E1
:10DE500013604FF030020A802BE04FF010030B806C
:10DE6000072626E0A68AA2699E4234BF35461D4693
:10DE70002846B34294BF0426022690470746002056
:10DE800000F060FD2A460146384600F069FB29464D
:10DE9000002000F073FD638A228AEB186382094B2D
:10DEA000551B4FF0300225821A80094B4FF4405227
:10DEB0001A80024B1B681E72F8BD00BF740C002054
:10DEC00040060020D80C0020505C004002300020AA
:10DED000D60C002008B5144B1B681A7A022A01D010
:10DEE000042A05D1FFF7A0FF0F4B1B681B7A14E033
:10DEF000062A11D15A78052A0AD11A7812F07F0F12
:10DF000006D1D878FFF7E2FE084B1B681B6A9847DA
:10DF1000074B1B689B6898470823034A12681372D3
:10DF2000FFF7F8FE08BD00BF740C0020300C002085
:10DF30000C0C002038B5324B1B68187810F07F00AD
:10DF400004D15A7A22F020025A7258E0022855D1A0
:10DF50005A88002A52D11A79002A4FD15A7912F0E0
:10DF6000800F22F0800405D0264951F8241001F0DA
:10DF7000300104E0234951F8241001F440512248B3
:10DF8000007884423AD2002938D09B7A002B35D0D1
:10DF900012F0800F0FD01B4B53F8243003F03003E6
:10DFA000102B25D1E4B2204600F082FC204630211F
:10DFB00000F05EFB1CE0134D55F8243003F4405391
:10DFC000B3F5805F14D134B9104B204693F82C1070
:10DFD00000F0F6FC02E0204600F056FC55F8242044
:10DFE0004BF68F7302EA030383F4405345F8243061
:10DFF000074B1B685B699847002000E0022038BD92
:10E00000740C0020005C0040000100207C00002017
:10E01000300C0020F7B58D4B8D4E1A6835688D4B4E
:10E0200092B2D3182A7A5B00092A1B681BD09BB2D4
:10E0300003F1005303F540535B001C4614F8012B19
:10E0400003F10A072A705B786B70B4F8030000F0E4
:10E0500063FE6880B4F80700346800F05DFEA080BD
:10E0600033687F88DF807A4C01212368DA8819724F
:10E070005D78002A62D11A7812F07F022ED1092D24
:10E0800002D1FFF715FD3BE0052D0DD193F90320DB
:10E09000002A4EDB9A78002A4BD19A88002A48D170
:10E0A0009B7A002B37D044E0032D0BD1DA78012A7C
:10E0B00027D19A882ABB5B7A13F0200F21D0FFF773
:10E0C000E5FD1DE0012D1CD1DA78012A19D19A88CD
:10E0D000BAB95B7A13F0200F13D00AE0012A04D1F9
:10E0E0000B2D0ED1FFF714FD0AE0022A09D1012DF4
:10E0F00002D1FFF71FFF03E0032D02D1FFF780FDE0
:10E1000048B1554B28461B685B699847032801D1E5
:10E1100009230FE068B94D4A504B12684FF03001A7
:10E1200092B2D3185B0000221A604D4B198006236F
:10E1300000E00823464A12681372E3E0062D18D166
:10E140001A7812F07F0F40F097809B78012B03D153
:10E15000414B1B68DB696EE0022B03D13E4B1B6811
:10E160001B6A68E0032B40F087803B4B1B685B6AAF
:10E1700061E0002D3CD1598800297DD15A6822F4F4
:10E180007F42B2F5003F77D11A7812F07F0203D1B7
:10E190009B88002B70D129E0012A0BD158792E4B96
:10E1A0001B689B699847002866D123689B7A002BDF
:10E1B00062D01BE0022A5FD15B7913F0800F03F07D
:10E1C0000F0205D0274951F8221001F0300104E078
:10E1D000244951F8221001F440512348007882422A
:10E1E0004AD213F0700F47D1002945D01F4B23E0CE
:10E1F000082D05D11B7813F07F0F3DD11C4B1BE080
:10E200000A2D39D11A7802F07F02012A34D19A7A84
:10E21000002A31D0598800292ED15A6822F47F4231
:10E22000B2F5803F28D158790B4B1B689B69984702
:10E2300010BB104B00E0FBB1054A4FF00001126823
:10E240000020936151829847002020E0505C0040FC
:10E25000740C0020043000200C0C00200230002040
:10E26000D80C0020005C00400001002059DB0008B1
:10E2700089DA0008E9DA0008244C254B22681B687B
:10E2800050781B699847032801D1236806E01F4B8B
:10E290004FF6FF711B681A8A8A4201D1092203E0F6
:10E2A000022800D012B908221A722BE093F900104C
:10E2B000002921DAD98801910198824202D9019A74
:10E2C0001A8211E08A420FD21149096891F82C1084
:10E2D0008A4201D2002105E092FBF1F001FB1022FD
:10E2E00012B901210B4A1170094A126892F82C20C8
:10E2F0009A82FFF799FD05E003221A72064B4FF44C
:10E3000040521A80FFF706FDFEBD00BF740C0020CE
:10E310000C0C002040060020D60C0020074A0221E9
:10E3200008B5074811720749074B086007490A609A
:10E33000074A13601B68984708BD00BF140C0020F3
:10E3400004010020300C00207C000020740C002010
:10E350000C0C002008B529E047F6FF70086019880A
:10E3600001F00F018B0003F18043117003F5B843F6
:10E37000196889B211F4004F09D0186840F68F71FE
:10E3800000EA0101196012780E4B013A0BE011F01E
:10E39000800F0BD0186848F60F7100EA0101196070
:10E3A0001278094B013A53F8223098470749084B35
:10E3B0000868084A80B21880188800B20028CBDBB1
:10E3C00008BD00BFE4000020C8000020445C0040FD
:10E3D0000A0C0020100C0020F8B59AE047F6FF76F2
:10E3E0001E601688564F06F00F06B30003F18043F7
:10E3F00003F5B8433E70002E64D127682668236871
:10E4000007F4405C03EA000080F4005020602368B9
:10E4100006F0300003EA010181F020012160138839
:10E42000484A13F0100F1080A5F800C004D02368EC
:10E430009BB213F0800F08D0226848F60F7302EAEF
:10E4400003032360FFF746FD16E013F4006F08D0C6
:10E45000226840F68F7302EA03032360FFF7DAFDB8
:10E460000AE013F4004F54D0226840F68F7302EA9A
:10E4700003032360FFF770FC21682A884BF68F7333
:10E4800001EA030312F4805F18BF83F4805312F48F
:10E49000005F2D4A18BF83F400531360294B1168A5
:10E4A0001A8848F6BF7301EA030312F0100F18BF71
:10E4B00083F0100312F0200F234A18BF83F02003CB
:10E4C00013603BE01C68A4B214F4004F0BD0196831
:10E4D00040F68F7201EA02021A603A781B4B013A49
:10E4E00053F82230984714F0800F12D0144948F6A0
:10E4F0000F720B789B0003F1804303F5B843186853
:10E5000000EA02021A600A78114B013A53F82230ED
:10E510009847104B104A1D680B4C1FFA85FCA2F857
:10E5200000C0B2F800C04BF68F700FFA8CFCBCF143
:10E53000000F48F6BF71094DFFF650AFF8BD00BFA0
:10E54000100C0020D80C0020005C0040E4000020EB
:10E55000C8000020445C00400A0C0020D60C0020BB
:10E5600001F10051013201F5405110B54900520846
:10E57000002308E010F803C06478013A4CEA042C48
:10E5800021F813C00233C418002AF3D110BD00BF14
:10E5900001F10051013201F5405110B54900520816
:10E5A000002304E031F81340013AC4520233002A38
:10E5B000F8D110BD014B1860704700BF405C0040AF
:10E5C000014B186880B27047405C0040014B1860F6
:10E5D000704700BF445C0040014B186880B2704730
:10E5E000445C0040014B186880B27047485C0040B2
:10E5F000014B1860704700BF4C5C0040014B18682D
:10E6000080B270474C5C00404FF6F873024A00EA53
:10E6100003031360704700BF505C0040014B186853
:10E6200080B27047505C0040014B43F820107047A7
:10E63000005C0040024B53F8200080B2704700BFDE
:10E64000005C0040054B10B553F8204048F68F128F
:10E6500004EA02020A4343F8202010BD005C004097
:10E66000024B53F8200000F4C0607047005C00408B
:10E670000A4B10B553F8202048F6BF7402EA040490
:10E6800011F0100F18BF84F0100411F0200F18BF04
:10E6900084F0200443F8204010BD00BF005C00401F
:10E6A0000A4B10B553F820204BF68F7402EA04048D
:10E6B00011F4805F18BF84F4805411F4005F18BF18
:10E6C00084F4005443F8204010BD00BF005C0040BB
:10E6D00038B50D460446FFF7ADFF012D02D120F4F9
:10E6E000805003E0022D04D120F01000014B43F8CC
:10E6F000240038BD005C0040024B53F8200000F0BD
:10E7000030007047005C0040024B53F8200000F4DA
:10E7100040507047005C0040054B48F6BF7253F80C
:10E72000201001EA020282F0300243F820207047F4
:10E73000005C0040054B4BF68F7253F8201001EA45
:10E74000020282F4405243F820207047005C0040EF
:10E75000054B48F68F6253F8201001EA020242F49A
:10E76000807243F820207047005C0040044B48F65C
:10E770008F6253F8201001EA020243F8202070470C
:10E78000005C0040044B48F68F6253F8201001EA09
:10E79000020243F820207047005C0040054B48F619
:10E7A0008F6253F8201001EA020242F4807243F8AB
:10E7B00020207047005C0040054B48F68F6253F8FC
:10E7C000201001EA020242F4807243F820207047D0
:10E7D000005C0040044B48F68F6253F8201001EAB9
:10E7E000020243F820207047005C0040044B53F8BD
:10E7F000200000F03000102814BF002001207047D6
:10E80000005C0040054B53F8200000F44050B0F588
:10E81000805F14BF00200120704700BF005C0040F3
:10E82000044B40F68F7253F8201001EA020243F8BD
:10E8300020207047005C0040044B48F60F7253F8EC
:10E84000201001EA020243F820207047005C0040DB
:10E85000054B48F68F7253F8201001EA020242F489
:10E86000804243F820207047005C0040054B48F68A
:10E870008F7253F8201001EA020242F0400243F87E
:10E8800020207047005C0040084B53F8202012F411
:10E89000804F09D053F8201048F68F7201EA020227
:10E8A00042F4804243F82020704700BF005C0040E3
:10E8B000084B53F8202012F0400F09D053F82010D5
:10E8C00048F68F7201EA020242F0400243F820202B
:10E8D000704700BF005C0040054B10B553F8204066
:10E8E00048F68F7204EA02020A4343F8202010BD62
:10E8F000005C0040024B53F8200000F00F0070470E
:10E90000005C0040064B49081B6849009BB203EBC2
:10E91000C00303F1005303F540535B0019607047D7
:10E92000505C0040054A064B1268490892B202EB5F
:10E93000C002D3185B00490019607047505C00406A
:10E9400004300020054B1B689BB203EBC00303F1AE
:10E95000005303F540535B0018887047505C00403B
:10E96000044A054B126892B202EBC002D3185B0056
:10E9700018887047505C004004300020044A054B62
:10E98000126892B202EBC002D3185B0019607047A4
:10E99000505C0040023000203E2909D94B0911F09B
:10E9A0001F0F01D1013B9BB29B0243F4004305E0E2
:10E9B0004B0811F0010F18BF01339B020360704731
:10E9C0000D4A0E4B126892B2D31803EBC0035B00E2
:10E9D0003E2909D94A0911F01F0F01D1013A92B21B
:10E9E000920242F4004205E04A0811F0010F18BFFC
:10E9F000013292021A607047505C004006300020DD
:10EA0000054A064B126892B202EBC002D3185B00B3
:10EA100018688005800D7047505C0040023000206F
:10EA2000054A064B126892B202EBC002D3185B0093
:10EA300018688005800D7047505C0040063000204B
:10EA40000C4B30B51D681C68C0001FFA85FC84445F
:10EA5000A4B2094B00190CF1005CC3180CF5405C22
:10EA6000490852084FEA4C0049005B00520001601F
:10EA70001A6030BD505C004004300020064B49084D
:10EA80001B6849009BB203EBC00303F1005303F57D
:10EA900040535B0019607047505C0040054A064BCC
:10EAA0001268490892B202EBC002D3185B00490019
:10EAB00019607047505C004004300020054B1B6813
:10EAC0009BB203EBC00303F1005303F540535B001B
:10EAD00018887047505C0040044A054B126892B297
:10EAE00002EBC002D3185B0018887047505C0040EE
:10EAF00004300020012910B524D1254B25491B687D
:10EB0000C0009BB2591809184B003E2A09D9510977
:10EB100012F01F0F01D1013989B2890241F400417D
:10EB200005E0510812F0010F18BF01318902196088
:10EB30001749194B096889B2CB18181840003E2AAA
:10EB40001ED913E0022922D1114BC0001C681B689A
:10EB5000A4B21FFA83FC0F490F4B844400194118DB
:10EB6000634449005B000A601A6010E0530912F028
:10EB70001F0F01D1013B9BB29B0243F4004305E010
:10EB8000530812F0010F18BF01339B02036010BD40
:10EB9000505C0040023000200630002001291BD1CB
:10EBA0001349144B096889B2CB1803EBC00040002D
:10EBB0003E2A09D9530912F01F0F01D1013B9BB224
:10EBC0009B0243F4004305E0530812F0010F18BF05
:10EBD00001339B0203600AE0022908D10449054B76
:10EBE000096889B201EBC000C3185B001A60704766
:10EBF000505C00400230002001291BD11349144B06
:10EC0000096889B2CB1803EBC00040003E2A09D93D
:10EC1000530912F01F0F01D1013B9BB29B0243F439
:10EC2000004305E0530812F0010F18BF01339B02A7
:10EC300003600AE0022908D10449054B096889B23A
:10EC400001EBC000C3185B001A607047505C0040C5
:10EC500006300020054A064B126892B202EBC00251
:10EC6000D3185B0018688005800D7047505C004029
:10EC700002300020054A064B126892B202EBC00235
:10EC8000D3185B0018688005800D7047505C004009
:10EC9000063000200D4BC00019680D4A89B241189A
:10ECA0008A185200128812F47C4F01D001200CE027
:10ECB0001A68084B92B28018C3185B001888800548
:10ECC000800D002814BF022000207047505C0040D7
:10ECD0000630002002300020012909D10B4A48F6F5
:10ECE0008F7352F8201001EA030343F040030AE057
:10ECF00002290AD1054A48F68F7352F8201001EA1A
:10ED0000030343F4804342F820307047005C004026
:10ED100041EA0020704700BF030AC0B243EA002066
:10ED2000704700BF08B500220A2300F045F808BD6F
:10ED300008B500210A2200F0DFF808BDF0B403781E
:10ED4000002B2DD040F23012C2F20002156802E012
:10ED500010F8013FEBB15A1903F12004527812F078
:10ED600001070A7808BF1C4601F10101561C9446B0
:10ED7000AE5D16F0010F18BF02F1200C6445E7D01C
:10ED800007B1203316F0010F18BF2032981AF0BCDB
:10ED900070470A786F78561C07F00107AE5DEFE701
:10EDA00040F230100A78C2F20000561C05686F78F5
:10EDB000AE5D07F00107E3E72DE9F04F40F23015B3
:10EDC000C2F2000583B00C461F46D5F800800E46FF
:10EDD0000190009216F8015B08EB050393F801B06F
:10EDE0001BF0080BF6D12D2D65D02B2D08BF16F882
:10EDF000015BD7F1010338BF0023102F14BF1A465F
:10EE000043F0010232B1302D66D01BB1302D0CBF62
:10EE100008270A27BBF1000F394614BF4FF00049FD
:10EE20006FF00049484600F0A5F948468A46394641
:10EE300000F072F800218C4608EB0502A5F13003C2
:10EE4000527812F0040F08D112F0030F20D012F004
:10EE5000010F14BF37235723EB1A9F4218DD844557
:10EE600094BF0022012252EAD1714FF0FF310CD140
:10EE7000844514BF002201225345D4BF002202F072
:10EE8000010212B907FB0C3C012116F8015BD3E724
:10EE9000B1F1FF3F14D0BBF1000F09D16046009BD8
:10EEA0001BB101B1741E009A146003B0BDE8F08F6D
:10EEB000CCF10000F3E716F8015B4FF0010B98E787
:10EEC000019ABBF1000F4FF0220314BF4FF0004036
:10EED0006FF000401360E2E73278782A14BF002117
:10EEE0000121582A14BF0A4641F00102002A8CD0A1
:10EEF0007578102702368DE710B540F23414C2F24F
:10EF000000048C461346014662462068FFF754FF12
:10EF100010BD00BF000000004A1E08BF7047C0F0CF
:10EF20002481884240F21681114200F01781B0FA24
:10EF300080F3B1FA81F2A2EB0303C3F11F0304A231
:10EF400002EB03134FF000029F4600BFAFF30080B7
:10EF5000B0EBC17F00BF42EB020228BFA0EBC17043
:10EF6000B0EB817F00BF42EB020228BFA0EB8170B3
:10EF7000B0EB417F00BF42EB020228BFA0EB417023
:10EF8000B0EB017F00BF42EB020228BFA0EB017093
:10EF9000B0EBC16F00BF42EB020228BFA0EBC16023
:10EFA000B0EB816F00BF42EB020228BFA0EB816093
:10EFB000B0EB416F00BF42EB020228BFA0EB416003
:10EFC000B0EB016F00BF42EB020228BFA0EB016073
:10EFD000B0EBC15F00BF42EB020228BFA0EBC15003
:10EFE000B0EB815F00BF42EB020228BFA0EB815073
:10EFF000B0EB415F00BF42EB020228BFA0EB4150E3
:10F00000B0EB015F00BF42EB020228BFA0EB015052
:10F01000B0EBC14F00BF42EB020228BFA0EBC140E2
:10F02000B0EB814F00BF42EB020228BFA0EB814052
:10F03000B0EB414F00BF42EB020228BFA0EB4140C2
:10F04000B0EB014F00BF42EB020228BFA0EB014032
:10F05000B0EBC13F00BF42EB020228BFA0EBC130C2
:10F06000B0EB813F00BF42EB020228BFA0EB813032
:10F07000B0EB413F00BF42EB020228BFA0EB4130A2
:10F08000B0EB013F00BF42EB020228BFA0EB013012
:10F09000B0EBC12F00BF42EB020228BFA0EBC120A2
:10F0A000B0EB812F00BF42EB020228BFA0EB812012
:10F0B000B0EB412F00BF42EB020228BFA0EB412082
:10F0C000B0EB012F00BF42EB020228BFA0EB0120F2
:10F0D000B0EBC11F00BF42EB020228BFA0EBC11082
:10F0E000B0EB811F00BF42EB020228BFA0EB8110F2
:10F0F000B0EB411F00BF42EB020228BFA0EB411062
:10F10000B0EB011F00BF42EB020228BFA0EB0110D1
:10F11000B0EBC10F00BF42EB020228BFA0EBC10061
:10F12000B0EB810F00BF42EB020228BFA0EB8100D1
:10F13000B0EB410F00BF42EB020228BFA0EB410041
:10F14000B0EB010F00BF42EB020228BFA0EB0100B1
:10F15000104670470CBF012000207047B1FA81F2C1
:10F16000C2F11F0220FA02F0704708B14FF0FF30E1
:10F1700000F00EB80029F8D02DE90340FFF7CCFECF
:10F18000BDE8064002FB00F3A1EB0301704700BF9E
:10F19000704700BF81F0004102E000BF83F00043F0
:10F1A00030B54FEA41044FEA430594EA050F08BF22
:10F1B00090EA020F1FBF54EA000C55EA020C7FEAE6
:10F1C000645C7FEA655C00F0E2804FEA5454D4EB63
:10F1D0005555B8BF6D420CDD2C4480EA020281EA2D
:10F1E000030382EA000083EA010180EA020281EA65
:10F1F0000303362D88BF30BD11F0004F4FEA0131B7
:10F200004FF4801C4CEA113102D0404261EB4101C5
:10F2100013F0004F4FEA03334CEA133302D052424B
:10F2200063EB430394EA050F00F0A780A4F1010407
:10F23000D5F1200E0DDB02FA0EFC22FA05F2801841
:10F2400041F1000103FA0EF2801843FA05F3594127
:10F250000EE0A5F120050EF1200E012A03FA0EFCA6
:10F2600028BF4CF0020C43FA05F3C01851EBE371D0
:10F2700001F0004507D54FF0000EDCF1000C7EEBED
:10F2800000006EEB0101B1F5801F1BD3B1F5001F2B
:10F290000CD349085FEA30004FEA3C0C04F101044A
:10F2A0004FEA445212F5800F80F09A80BCF1004F73
:10F2B00008BF5FEA500C50F1000041EB045141EAF5
:10F2C000050130BD5FEA4C0C404141EB010111F4F6
:10F2D000801FA4F10104E9D191F0000F04BF0146A1
:10F2E0000020B1FA81F308BF2033A3F10B03B3F17F
:10F2F00020020CDA0C3208DD02F1140CC2F10C020F
:10F3000001FA0CF021FA02F10CE002F11402D8BF6C
:10F31000C2F1200C01FA02F120FA0CFCDCBF41EA38
:10F320000C019040E41AA2BF01EB0451294330BD07
:10F330006FEA04041F3C1CDA0C340EDC04F11404E4
:10F34000C4F1200220FA04F001FA02F340EA0300BB
:10F3500021FA04F345EA030130BDC4F10C04C4F101
:10F36000200220FA02F001FA04F340EA03002946E1
:10F3700030BD21FA04F0294630BD94F0000F83F42B
:10F38000801306BF81F480110134013D4EE77FEA0E
:10F39000645C18BF7FEA655C29D094EA050F08BF5A
:10F3A00090EA020F05D054EA000C04BF194610463B
:10F3B00030BD91EA030F1EBF0021002030BD5FEA7F
:10F3C000545C05D14000494128BF41F0004130BDA7
:10F3D00014F580043CBF01F5801130BD01F00045FB
:10F3E00045F0FE4141F470014FF0000030BD7FEA6E
:10F3F000645C1ABF194610467FEA655C1CBF0B4669
:10F40000024650EA013406BF52EA033591EA030F7F
:10F4100041F4002130BD00BF90F0000F04BF002177
:10F42000704730B54FF4806404F132044FF00005AA
:10F430004FF0000150E700BF90F0000F04BF002123
:10F44000704730B54FF4806404F1320410F0004589
:10F4500048BF40424FF000013EE700BF42004FEA84
:10F46000E2014FEA31014FEA02701FBF12F07F4301
:10F4700093F07F4F81F06051704792F0000F14BFFE
:10F4800093F07F4F704730B54FF4607401F0004542
:10F4900021F0004120E700BF50EA010208BF704799
:10F4A00030B54FF000050AE050EA010208BF70478E
:10F4B00030B511F0004502D5404261EB41014FF4F7
:10F4C000806404F132045FEA915C3FF4DCAE4FF0FB
:10F4D00003025FEADC0C18BF03325FEADC0C18BFE2
:10F4E000033202EBDC02C2F1200300FA03FC20FA33
:10F4F00002F001FA03FE40EA0E0021FA02F1144480
:10F50000C1E600BF70B54FF0FF0C4CF4E06C1CEA94
:10F5100011541DBF1CEA135594EA0C0F95EA0C0F09
:10F5200000F0DEF82C4481EA030621EA4C5123EA7C
:10F530004C5350EA013518BF52EA033541F48011AB
:10F5400043F4801338D0A0FB02CE4FF00005E1FB5E
:10F5500002E506F00042E0FB03E54FF00006E1FBA8
:10F5600003569CF0000F18BF4EF0010EA4F1FF04EB
:10F57000B6F5007F64F5407404D25FEA4E0E6D412B
:10F5800046EB060642EAC62141EA55514FEAC5203C
:10F5900040EA5E504FEACE2EB4F1FD0C88BFBCF5B8
:10F5A000E06F1ED8BEF1004F08BF5FEA500E50F169
:10F5B000000041EB045170BD06F0004646EA01012F
:10F5C00040EA020081EA0301B4EB5C04C2BFD4EB61
:10F5D0000C0541EA045170BD41F480114FF0000E5A
:10F5E000013C00F3AB8014F1360FDEBF002001F0C8
:10F5F000004170BDC4F10004203C35DA0C341BDC42
:10F6000004F11404C4F1200500FA05F320FA04F013
:10F6100001FA05F240EA020001F0004221F0004147
:10F6200010EBD37021FA04F642EB06015EEA430EBA
:10F6300008BF20EAD37070BDC4F10C04C4F12005EA
:10F6400000FA04F320FA05F001FA04F240EA02009D
:10F6500001F0004110EBD37041F100015EEA430E6E
:10F6600008BF20EAD37070BDC4F1200500FA05F28E
:10F670004EEA020E20FA04F301FA05F243EA02030D
:10F6800021FA04F001F0004121FA04F220EA02001C
:10F6900000EBD3705EEA430E08BF20EAD37070BD62
:10F6A00094F0000F0FD101F00046400041EB010142
:10F6B00011F4801F08BF013CF7D041EA060195F024
:10F6C000000F18BF704703F00046520043EB0303DE
:10F6D00013F4801F08BF013DF7D043EA06037047CB
:10F6E00094EA0C0F0CEA135518BF95EA0C0F0CD0D6
:10F6F00050EA410618BF52EA4306D1D181EA03011C
:10F7000001F000414FF0000070BD50EA410606BF15
:10F710001046194652EA430619D094EA0C0F02D15A
:10F7200050EA013613D195EA0C0F05D152EA03369F
:10F730001CBF104619460AD181EA030101F00041BD
:10F7400041F0FE4141F470014FF0000070BD41F006
:10F75000FE4141F4780170BD70B54FF0FF0C4CF4E0
:10F76000E06C1CEA11541DBF1CEA135594EA0C0FFF
:10F7700095EA0C0F00F0A7F8A4EB050481EA030E4C
:10F7800052EA03354FEA013100F088804FEA033333
:10F790004FF0805545EA131343EA12634FEA022201
:10F7A00045EA111545EA10654FEA00260EF00041C2
:10F7B0009D4208BF964244F1FD0404F5407402D214
:10F7C0005B084FEA3202B61A65EB03055B084FEAA5
:10F7D00032024FF480104FF4002CB6EB020E75EBA2
:10F7E000030E22BFB61A754640EA0C005B084FEACA
:10F7F0003202B6EB020E75EB030E22BFB61A754647
:10F8000040EA5C005B084FEA3202B6EB020E75EB91
:10F81000030E22BFB61A754640EA9C005B084FEA09
:10F820003202B6EB020E75EB030E22BFB61A754616
:10F8300040EADC0055EA060E18D04FEA051545EA05
:10F8400016754FEA06164FEAC30343EA52734FEAAE
:10F85000C2025FEA1C1CC0D111F4801F0BD141EA27
:10F8600000014FF000004FF0004CB6E711F4801F8C
:10F8700004BF01430020B4F1FD0C88BFBCF5E06F6C
:10F880003FF6AFAEB5EB030C04BFB6EB020C5FEA7C
:10F89000500C50F1000041EB045170BD0EF0004ED1
:10F8A0004EEA113114EB5C04C2BFD4EB0C0541EA03
:10F8B000045170BD41F480114FF0000E013C90E600
:10F8C00045EA060E8DE60CEA135594EA0C0F08BFC4
:10F8D00095EA0C0F3FF43BAF94EA0C0F0AD150EAC3
:10F8E00001347FF434AF95EA0C0F7FF425AF104656
:10F8F00019462CE795EA0C0F06D152EA03353FF47E
:10F90000FDAE1046194622E750EA410618BF52EAFA
:10F9100043067FF4C5AE50EA41047FF40DAF52EACE
:10F9200043057FF4EBAE12E74FEA410212F50012F5
:10F9300015D211D56FF47873B3EB625212D94FEA36
:10F94000C12343F0004343EA505311F0004F23FA20
:10F9500002F018BF404270474FF00000704750EA75
:10F96000013005D111F0004008BF6FF00040704732
:10F970004FF00000704700BF4FEA4102B2F1E04390
:10F9800024BFB3F5001CDCF1FE5C0DD901F0004C86
:10F990004FEAC0024CEA5070B2F1004F40EB8300D6
:10F9A00008BF20F00100704711F0804F21D113F102
:10F9B0003872BCBF01F00040704741F480114FEA3B
:10F9C0005252C2F11802C2F1200C10FA0CF320FAC4
:10F9D00002F018BF40F001004FEAC1234FEAD323E1
:10F9E00003FA0CFC40EA0C0023FA02F34FEA43034B
:10F9F000CCE77FEA625307D150EA01331EBF4FF0D4
:10FA0000FE4040F44000704701F0004040F0FE40EE
:10FA100040F40000704700BF80F0004002E000BFEB
:10FA200081F0004142001FBF5FEA410392EA030FE9
:10FA30007FEA226C7FEA236C6AD04FEA1262D2EB33
:10FA40001363C1BFD218414048404140B8BF5B4238
:10FA5000192B88BF704710F0004F40F4000020F0D1
:10FA60007F4018BF404211F0004F41F4000121F0E7
:10FA70007F4118BF494292EA030F3FD0A2F1010231
:10FA800041FA03FC10EB0C00C3F1200301FA03F16F
:10FA900000F0004302D5494260EB4000B0F5000F92
:10FAA00013D3B0F1807F06D340084FEA310102F151
:10FAB0000102FE2A51D2B1F1004F40EBC25008BF03
:10FAC00020F0010040EA03007047490040EB0000CD
:10FAD00010F4000FA2F10102EDD1B0FA80FCACF1FC
:10FAE000080CB2EB0C0200FA0CF0AABF00EBC250FB
:10FAF00052421843BCBFD0401843704792F0000FE9
:10FB000081F4000106BF80F400000132013BB5E73B
:10FB10004FEA41037FEA226C18BF7FEA236C21D0B1
:10FB200092EA030F04D092F0000F08BF0846704716
:10FB300090EA010F1CBF0020704712F07F4F04D1E4
:10FB4000400028BF40F00040704712F100723CBFF7
:10FB500000F50000704700F0004343F0FE4040F421
:10FB6000000070477FEA226216BF08467FEA2363DF
:10FB70000146420206BF5FEA412390EA010F40F4CA
:10FB8000800070474FF0000304E000BF10F0004316
:10FB900048BF40425FEA000C08BF704743F09643FD
:10FBA00001464FF000001CE050EA010208BF704718
:10FBB0004FF000030AE000BF50EA010208BF70479F
:10FBC00011F0004302D5404261EB41015FEA010CB4
:10FBD00002BF84460146002043F0B64308BFA3F1AC
:10FBE0008053A3F50003BCFA8CF2083AA3EBC2538E
:10FBF00010DB01FA02FC634400FA02FCC2F12002AD
:10FC0000BCF1004F20FA02F243EB020008BF20F0E3
:10FC10000100704702F1200201FA02FCC2F1200249
:10FC200050EA4C0021FA02F243EB020008BF20EA3E
:10FC3000DC7070474FF0FF0C1CEAD0521EBF1CEA6C
:10FC4000D15392EA0C0F93EA0C0F6FD01A4480EA5A
:10FC5000010C400218BF5FEA41211ED04FF0006343
:10FC600043EA501043EA5111A0FB01310CF000406F
:10FC7000B1F5000F3EBF490041EAD3715B0040EA95
:10FC8000010062F17F02FD2A1DD8B3F1004F40EB65
:10FC9000C25008BF20F00100704790F0000F0CF038
:10FCA000004C08BF49024CEA502040EA51207F3AFC
:10FCB000C2BFD2F1FF0340EAC250704740F40000D7
:10FCC0004FF00003013A5DDC12F1190FDCBF00F0C8
:10FCD00000407047C2F10002410021FA02F1C2F176
:10FCE000200200FA02FC5FEA310040F1000053EA12
:10FCF0004C0308BF20EADC70704792F0000F00F060
:10FD0000004C02BF400010F4000F013AF9D040EA65
:10FD10000C0093F0000F01F0004C02BF490011F4F9
:10FD2000000F013BF9D041EA0C018FE70CEAD153F7
:10FD300092EA0C0F18BF93EA0C0F0AD030F0004C77
:10FD400018BF31F0004CD8D180EA010000F000402B
:10FD5000704790F0000F17BF90F0004F084691F0E9
:10FD6000000F91F0004F14D092EA0C0F01D1420223
:10FD70000FD193EA0C0F03D14B0218BF084608D1EC
:10FD800080EA010000F0004040F0FE4040F4000036
:10FD9000704740F0FE4040F4400070474FF0FF0CC9
:10FDA0001CEAD0521EBF1CEAD15392EA0C0F93EA10
:10FDB0000C0F69D0A2EB030280EA010C49024FEA62
:10FDC000402037D04FF0805343EA111143EA10131B
:10FDD0000CF000408B4238BF5B0042F17D024FF4D3
:10FDE000000C8B4224BF5B1A40EA0C00B3EB510FAE
:10FDF00024BFA3EB510340EA5C00B3EB910F24BF97
:10FE0000A3EB910340EA9C00B3EBD10F24BFA3EB1B
:10FE1000D10340EADC001B0118BF5FEA1C1CE0D1E3
:10FE2000FD2A3FF650AF8B4240EBC25008BF20F096
:10FE3000010070470CF0004C4CEA50207F32C2BFEA
:10FE4000D2F1FF0340EAC250704740F400004FF087
:10FE50000003013A37E792F0000F00F0004C02BFB8
:10FE6000400010F4000F013AF9D040EA0C0093F082
:10FE7000000F01F0004C02BF490011F4000F013BDC
:10FE8000F9D041EA0C0195E70CEAD15392EA0C0F44
:10FE900008D142027FF47DAF93EA0C0F7FF470AF7C
:10FEA000084676E793EA0C0F04D14B023FF44CAFBF
:10FEB00008466EE730F0004C18BF31F0004CCAD154
:10FEC00030F000427FF45CAF31F000437FF43CAF90
:10FED0005FE700BF4FF0FF3C06E000BF4FF0010CB2
:10FEE00002E000BF4FF0010C4DF804CD4FEA400294
:10FEF0004FEA41037FEA226C18BF7FEA236C11D0DE
:10FF000001B052EA530C18BF90EA010F58BFB2EB90
:10FF1000030088BFC81738BF6FEAE17018BF40F010
:10FF2000010070477FEA226C02D15FEA402C05D1C4
:10FF30007FEA236CE4D15FEA412CE1D05DF8040B49
:10FF4000704700BF844608466146FFE70FB5FFF7DC
:10FF5000C9FF002848BF10F1000F0FBD4DF808ED94
:10FF6000FFF7F4FF0CBF012000205DF808FB00BF85
:10FF70004DF808EDFFF7EAFF34BF012000205DF8DF
:10FF800008FB00BF4DF808EDFFF7E0FF94BF01202C
:10FF900000205DF808FB00BF4DF808EDFFF7D2FF29
:10FFA00094BF012000205DF808FB00BF4DF808ED6C
:10FFB000FFF7C8FF34BF012000205DF808FB00BF39
:10FFC00042000ED2B2F1FE4F0BD34FF09E03B3EBC3
:10FFD000126209D44FEA002343F0004323FA02F0EF
:10FFE00070474FF00000704712F1610F01D14202DB
:10FFF00002D14FF0FF3070474FF00000704700BF54
:020000040801F1
:100000000000000000000000010003E80000000004
:1000100000000003E800000000000200FA060003F0
:100020000000000000370600000000000000000093
:10003000F4010000640000000180080800000000D6
:10004000000200000000000000000000C8000000E6
:100050001201100102000040D016A0050114010297
:100060000301000009024300020100C0320904003C
:100070000001020201000524001001052401000115
:10008000042402020524060001070582030800FF7C
:1000900009040100020A00000007050302400000F5
:1000A00007058102400000000403090426035400F0
:1000B000720069006E0061006D00690063004D0010
:1000C0006F00740069006F006E0020004300740030
:1000D0006C000000320354004D0043004D002D0021
:1000E0003100310034003100200028007600690022
:1000F00072007400750061006C00200043004F0026
:100100004D00290020000000524F5200000106520D
:100110004F4C000002064D5354000003024D565050
:1001200000000407534150000005074741500000FC
:100130000603535441500007035253415000080333
:100140005347500000090747475000000A03535423
:100150004750000B0352534750000C0352465300C4
:10016000000D0353494F00000E0747494F00000F91
:100170000353414300001D0753434F00001E074730
:10018000434F00001F0343434F0000200341434FF0
:100190000000270355463000004007554631000057
:1001A00041075546320000420755463300004307D9
:1001B000554634000044075546350000450755466E
:1001C00036000046075546370000470752554E0097
:1001D00000810553544F5000800042494E00008B6F
:1001E0000000000000000000000000000102030405
:1001F0000102030406070809020406080020202063
:1002000020202020202028282828282020202020C6
:100210002020202020202020202020202088101096
:1002200010101010101010101010101010040404F2
:1002300004040404040404101010101010104141B0
:10024000414141410101010101010101010101019E
:1002500001010101010101011010101010104242B2
:10026000424242420202020202020202020202026E
:10027000020202020202020210101010200000000E
:10028000000000000000000000000000000000006E
:10029000000000000000000000000000000000005E
:1002A000000000000000000000000000000000004E
:1002B000000000000000000000000000000000003E
:1002C000000000000000000000000000000000002E
:1002D000000000000000000000000000000000001E
:1002E000000000000000000000000000000000000E
:1002F00000000000000000000000000000000000FE
:100300003131343156313230004142530052454C84
:1003100000434F4F52440053544152540053544FE2
:100320005000535441545553000000004300000056
:1003300000030108000102000008000001000000A5
:1003400002000000000000000000000000000000AB
:10035000000000000000000000000000000000009D
:10036000000000000000000000000000000000008D
:100370000000000000C2010000000800A800010801
:1003800004000000AC00010826000000D4000108B1
:1003900032000000AC0000201A00000064000108D8
:1003A000430000005000010812000000A18A00086C
:1003B000AD880008BD860008D1860008D5860008F3
:1003C00035870008598700089D8800088D88000837
:1003D0006988000800000000400000001A03540073
:1003E0004D004300310031003400310000000000B6
:1003F0000000000000000000BD85000811DD0008BD
:1004000011DD000811DD000811DD000811DD000814
:1004100011DD000811DD000811DD0008FD8900086C
:1004200011DD000811DD000811DD000811DD0008F4
:100430000401000011DD00089986000811DD0008A4
:1004400011DD000811DD000811DD000811DD0008D4
:1004500011DD0008B186000801000000FD0101085F
:10046000FC0101083801002000000000000000002D
:10047000000000000000000000000000000000007C
:1004800000000000000000002C0301080000000034
:10049000000000000000000000000000000000005C
:1004A000000000000000000000000000000000004C
:1004B000000000000000000000000000000000003C
:1004C000000000000000000000000000000000002C
:1004D000000000000000000000000000000000001C
:1004E000000000000000000000000000000000000C
:1004F00000000000000000000000000000000000FC
:1005000000000000000000000000000000000000EB
:1005100000000000000000000000000000000000DB
:1005200000000000000000000000000000000000CB
:1005300000000000000000000000000000000000BB
:1005400000000000000000000000000000000000AB
:080550000000000000000000A3
:04000005080041109E
:00000001FF
